:100000000C94501A0C946D1A0C946D1A0C94301DAB
:100010000C946D1A0C946D1A0C946D1A0C94102992
:100020000C946D1A0C946D1A0C946D1A0C946D1A34
:100030000C946D1A0C94251B0C946D1A0C946D1A6B
:100040000C946D1A0C946D1A0C946D1A0C946D1A14
:100050000C946D1A4552524F520D0A0D0A0052650A
:100060006164790D0A0D0A000D0A00436F6D706915
:100070006C69657274206D6974204743432056652E
:100080007273696F6E20342E322E32202857696EBB
:10009000415652203230303731323231290D0A0088
:1000A000436F6D70696C6965727420616D20536572
:1000B00070203235203230303820756D2032333A9E
:1000C00035353A34380D0A000A0D53797374656D6D
:1000D0002052656164790A0D003A20504F4E472145
:1000E0000D0A002E2569002E2569002E25690025A0
:1000F00069004D792049503A202531692E25316912
:100100002E2531692E2531690D0A0D0A005245410F
:100110004459210D0A000A0D4E494320696E697445
:100120003A00524553455420202D20726573657462
:100130002074686520415652202D20436F6E7472E2
:100140006F6C6C65720D0A415250202020202D20CA
:100150006C69737420746865204152502074616228
:100160006C650D0A544350202020202D206C6973AB
:10017000742074686520746370207461626C650D0E
:100180000A495020202020202D206C6973742F6391
:1001900068616E67652069700D0A4E455420202005
:1001A000202D206C6973742F6368616E6765206E03
:1001B00065746D61736B0D0A524F55544552202D75
:1001C000206C6973742F6368616E676520726F7548
:1001D0007465722069700D0A4E5450202020202D25
:1001E000206C6973742F6368616E6765204E54508C
:1001F0000D0A4E5450522020202D204E5450205293
:100200006566726573680D0A4D4143202020202DDC
:10021000206C697374204D41432D61646472657371
:10022000730D0A564552202020202D206C697374CE
:1002300020656E632076657273696F6E206E756DD2
:100240006265720D0A535620202020202D207365F0
:1002500074207661726961626C650D0A50494E477F
:100260002020202D2073656E642050696E670D0A72
:1002700054494D452020202D206765742074696DF8
:10028000650D0A48454C502020202D207072696E63
:10029000742048656C70746578740D0A3F202020C6
:1002A0002020202D207072696E742048656C707457
:1002B0006578740D0A002563000A0D54494D453ACE
:1002C000202532693A2532693A2532690D0A0049FA
:1002D0006E68616C74206465722056617269616237
:1002E0006C655B2532695D203D202532690D0A0071
:1002F000202054696D653A2534690D0A002020508C
:100300004F52543A253469002E253369002E253387
:1003100069002E25336900202049503A25336900B1
:1003200025326900202054696D653A2534690D0A2B
:10033000002E253369002E253369002E25336900F0
:10034000202049503A253369002E253278002E2589
:100350003278002E253278002E253278002E253274
:10036000780025326920204D41433A2532780045F6
:100370004E4332384A36302D56657273696F6E3A85
:10038000202531780D0A004D79204D41433A202532
:1003900032783A2532783A2532783A2532783A2539
:1003A00032783A2532780D0A00526F7574657220E2
:1003B00049503A202531692E2531692E2531692E83
:1003C0002531690D0A004E45544D41534B3A2025C5
:1003D00031692E2531692E2531692E2531690D0AA5
:1003E000004E54505F5365727665723A202531692C
:1003F0002E2531692E2531692E2531690D0A004DD2
:10040000792049503A202531692E2531692E253130
:10041000692E2531690D0A0041424344454647484B
:10042000494A4B4C4D4E4F505152535455565758C4
:10043000595A6162636465666768696A6B6C6D6E60
:100440006F707172737475767778797A3031323370
:100450003435363738392B2F3D000400051A06FF96
:10046000071F080009000AFF0B19C100C00DC232A6
:10047000CAEECB05C412C612C70CE400E520E21890
:10048000E3B1E015E16F3C686561643E3C6D657405
:100490006120687474702D65717569763D22436FB3
:1004A0006E74656E742D547970652220636F6E745E
:1004B000656E743D22746578742F68746D6C3B2092
:1004C000636861727365743D69736F2D38383539AF
:1004D0002D3122202F3E0D0A3C7469746C653E500C
:1004E0006F6C6C696E204156522D4E45542D494F0C
:1004F000205765627365727665723C2F7469746CFF
:10050000653E0D0A3C7374796C6520747970653DA5
:1005100022746578742F637373223E0D0A3C212D7B
:100520002D0D0A424F4459207B096D617267696E37
:100530003A20302030203020303B206261636B67EE
:10054000726F756E642D636F6C6F723A2077686995
:1005500074653B20746578742D616C69676E3A63CD
:10056000656E7465723B207D0D0A502C20444956FF
:100570002C2048312C204832207B666F6E742D660B
:10058000616D696C793A2076657264616E612C20C8
:10059000617269616C3B20666F6E742D73697A6558
:1005A0003A20313170783B7D0D0A4831207B202084
:1005B0006261636B67726F756E642D636F6C6F72CF
:1005C0003A20234343434346463B207061646469B9
:1005D0006E672D746F703A3570783B20706164647B
:1005E000696E672D626F74746F6D3A3570783B6613
:1005F0006F6E742D73697A653A20323070783B20C3
:10060000636F6C6F723A20233030343036303B20C9
:10061000666F6E742D7765696768743A626F6C6493
:100620003B206C65747465722D73706163696E67CD
:100630003A203870783B626F726465722D746F7007
:100640003A2032707820736F6C69642023454545E9
:100650004545453B20626F726465722D6C6566741A
:100660003A2032707820736F6C69642023454545C9
:100670004545453B626F726465722D626F74746F9D
:100680006D3A2032707820736F6C696420233030AB
:10069000343036303B20626F726465722D72696748
:1006A00068743A2032707820736F6C69642023304C
:1006B00030343036303B7D0D0A4832207B20666F67
:1006C0006E742D73697A653A20313570783B2070ED
:1006D000616464696E672D746F703A20323070788F
:1006E0003B2070616464696E672D6C6566743A3591
:1006F0003070783B2070616464696E672D72696741
:1007000068743A353070783B636F6C6F723A23309F
:1007100030343038303B20666F6E742D77656967F2
:1007200068743A626F6C643B20746578742D6465FC
:10073000636F726174696F6E3A756E6465726C692D
:100740006E653B626F726465722D746F703A203112
:10075000707820736F6C6964202330303430383007
:100760003B7D20502C2048312C204832207B6D616D
:100770007267696E3A20307078203070782035705A
:1007800078203070783B7D0D0A2D2D3E0D0A3C2FD0
:100790007374796C653E3C2F686561643E0D0A3C5C
:1007A000626C6F636B71756F74653E0D0A3C626CB1
:1007B0006F636B71756F74653E0D0A3C626F64798F
:1007C0003E3C64697620616C69676E3D2263656EAC
:1007D000746572223E0D0A3C68313E506F6C6C6944
:1007E0006E204156522D4E45542D494F205765627B
:1007F00073657276657220323030383C2F68313E36
:100800000D0A3C2F6469763E3C42523E0D0A3C681C
:10081000323E476C2675756D6C3B636B77756E73F6
:1008200063683C2F68323E3C42523E0D0A3C6831C0
:100830003E7A756D204765627572747374616720C6
:100840003C2F703E3C42523E0D0A3C703E44657265
:1008500020576562736572766572206C2661756DCE
:100860006C3B75667420212121203C2F703E3C4258
:10087000523E0D0A3C666F726D206E616D653D22C1
:10088000666F726D3122206D6574686F643D2270F1
:100890006F73742220616374696F6E3D22223E0D76
:1008A0000A3C7020616C69676E3D226C656674223B
:1008B0003E266E6273703B202020203C2F703E0D40
:1008C0000A3C7020616C69676E3D226C656674221B
:1008D0003E0D0A3C7020616C69676E3D226C656656
:1008E00074223E45696E67616265203D20504F521B
:1008F000542028616E2F61757329200D0A3C7020E9
:10090000616C69676E3D226C656674223E0D0A3C1F
:10091000696E70757420747970653D2263686563D3
:100920006B626F7822206E616D653D224F555422B7
:100930002076616C75653D2241222025504F52542E
:1009400043303E0D0A3C7370616E20636C617373BB
:100950003D225374696C32223E506F7274204320E2
:1009600050696E20303C2F7370616E3E3C2F703E9C
:100970000D0A3C7020616C69676E3D226C6566747F
:10098000223E0D0A3C696E70757420747970653D65
:1009900022636865636B626F7822206E616D653DCE
:1009A000224F5554222076616C75653D22422220EB
:1009B00025504F525443313E0D0A3C7370616E20F6
:1009C000636C6173733D225374696C32223E506FC5
:1009D000727420432050696E20313C2F7370616E19
:1009E0003E3C2F703E0D0A3C7020616C69676E3D85
:1009F000226C656674223E0D0A3C696E7075742027
:100A0000747970653D22636865636B626F7822203C
:100A10006E616D653D224F5554222076616C75657F
:100A20003D2243222025504F525443323E0D0A3C72
:100A30007370616E20636C6173733D225374696CD3
:100A400032223E506F727420432050696E20323C37
:100A50002F7370616E3E3C2F703E0D0A3C646976C8
:100A600020616C69676E3D226C656674223E0D0ADA
:100A70003C696E70757420747970653D2263686599
:100A8000636B626F7822206E616D653D224F555415
:100A9000222076616C75653D2244222025504F52FC
:100AA0005443333E0D0A3C7370616E20636C617376
:100AB000733D225374696C32223E506F727420432E
:100AC0002050696E20333C2F7370616E3E3C2F7056
:100AD0003E0D0A3C64697620616C69676E3D226C4C
:100AE000656674223E0D0A3C696E707574207479D7
:100AF00070653D22636865636B626F7822206E616A
:100B00006D653D224F5554222076616C75653D22FE
:100B100045222025504F525443343E0D0A3C7370F9
:100B2000616E20636C6173733D225374696C322271
:100B30003E506F727420432050696E20343C2F73F6
:100B400070616E3E3C2F703E0D0A3C6469762061F8
:100B50006C69676E3D226C656674223E0D0A3C69C5
:100B60006E70757420747970653D22636865636B7F
:100B7000626F7822206E616D653D224F55542220B0
:100B800076616C75653D2246222025504F525443B4
:100B9000353E0D0A3C7370616E20636C6173733D6A
:100BA000225374696C32223E506F7274204320507D
:100BB000696E20353C2F7370616E3E3C2F703E0D88
:100BC0000A3C64697620616C69676E3D226C6566DB
:100BD00074223E0D0A3C696E7075742074797065DC
:100BE0003D22636865636B626F7822206E616D657C
:100BF0003D224F5554222076616C75653D22472277
:100C00002025504F525443363E0D0A3C7370616E9E
:100C100020636C6173733D225374696C32223E50C1
:100C20006F727420432050696E20363C2F737061C0
:100C30006E3E3C2F703E0D0A3C64697620616C6903
:100C4000676E3D226C656674223E0D0A3C696E70CB
:100C5000757420747970653D22636865636B626F9B
:100C60007822206E616D653D224F555422207661B9
:100C70006C75653D2248222025504F525443373E23
:100C80000D0A3C7370616E20636C6173733D225377
:100C900074696C32223E506F727420432050696E2A
:100CA00020373C2F7370616E3E3C2F703E0D0A3C26
:100CB00064697620616C69676E3D226C656674229A
:100CC0003E0D0A3C70726520616C69676E3D226C56
:100CD000656674223E3C696E707574207479706527
:100CE0003D227375626D697422206E616D653D22CF
:100CF000535542222076616C75653D2253656E64C2
:100D0000656E223E3C2F7072653E0D0A3C62723E5B
:100D10000D0A3C62723E0D0A3C703E20506F7274A8
:100D20002043202D204C454420416E7A656967653B
:100D30003C703E3C696D67207372633D22255049CB
:100D40004E4330222077696474683D223137222077
:100D50006865696768743D223137223E20506F72A2
:100D60007420412050696E20303C2F703E0D0A3CAB
:100D7000703E3C696D67207372633D222550494E79
:100D80004331222077696474683D2231372220681C
:100D900065696768743D223137223E20506F727456
:100DA00020412050696E20313C2F703E0D0A3C706E
:100DB0003E3C696D67207372633D222550494E4366
:100DC00032222077696474683D22313722206865B9
:100DD000696768743D223137223E20506F7274205B
:100DE000412050696E20323C2F703E0D0A3C703E0F
:100DF0003C696D67207372633D222550494E433331
:100E0000222077696474683D223137222068656941
:100E10006768743D223137223E20506F7274204142
:100E20002050696E20333C2F703E0D0A3C703E3CD2
:100E3000696D67207372633D222550494E43342209
:100E40002077696474683D223137222068656967BC
:100E500068743D223137223E20506F727420412049
:100E600050696E20343C2F703E0D0A3C703E3C6948
:100E70006D67207372633D222550494E4335222011
:100E800077696474683D2231372220686569676834
:100E9000743D223137223E20506F72742041205021
:100EA000696E20353C2F703E0D0A3C703E3C696DEA
:100EB00067207372633D222550494E4336222077C6
:100EC000696474683D2231372220686569676874F7
:100ED0003D223137223E20506F72742041205069EC
:100EE0006E20363C2F703E0D0A3C703E3C696D67AB
:100EF000207372633D222550494E43372220776983
:100F00006474683D22313722206865696768743DE2
:100F1000223137223E20506F727420412050696E7A
:100F200020373C2F703E0D0A3C62723E0D0A3C7425
:100F300061626C6520616C69676E3D2263656E74E9
:100F40006572222077696474683D22353030222032
:100F5000626F726465723D2230223E0D0A3C7472EB
:100F60003E0D0A3C74682073636F70653D22636FA9
:100F70006C223E3C7020616C69676E3D2263656E39
:100F8000746572223E45696E67616E673C2F703EE4
:100F90003C2F74683E0D0A3C74682073636F706563
:100FA0003D22636F6C223E3C7020616C69676E3D30
:100FB0002263656E746572223E42616C6B656E3CA5
:100FC0002F703E3C2F74683E0D0A3C74682073639A
:100FD0006F70653D22636F6C223E3C7020616C69CE
:100FE000676E3D2263656E746572223E54656D7056
:100FF000657261747572205B266465673B435D3C76
:101000002F703E3C2F74683E0D0A3C2F74723E0DCB
:101010000A3C74723E0D0A3C74643E3C7020616C64
:1010200069676E3D2263656E746572223E41442D90
:101030004B616E616C303C2F703E3C2F74643E0DF2
:101040000A3C74643E3C7020616C69676E3D2263AB
:10105000656E746572223E3C2F703E3C696D672060
:101060007372633D2262616C6B652E676966222034
:1010700077696474683D22255641403030222068EB
:1010800065696768743D223130223E3C2F74643EAE
:101090000D0A3C74643E3C7020616C69676E3D22B1
:1010A00063656E746572223E2556414030303C2F98
:1010B000703E3C2F74643E0D0A3C2F74723E0D0A44
:1010C0003C74723E0D0A3C74643E3C7020616C6955
:1010D000676E3D2263656E746572223E41442D4BFE
:1010E000616E616C313C2F703E3C2F74643E0D0A82
:1010F0003C74643E3C7020616C69676E3D226365A0
:101100006E746572223E3C2F703E3C696D672073A1
:1011100072633D2262616C6B652E6769662220777F
:10112000696474683D22255641403031222068654B
:10113000696768743D223130223E3C2F74643E0D55
:101140000A3C74643E3C7020616C69676E3D2263AA
:10115000656E746572223E2556414030313C2F70D9
:101160003E3C2F74643E0D0A3C2F74723E0D0A3CC7
:1011700074723E0D0A3C74643E3C7020616C696779
:101180006E3D2263656E746572223E41442D4B6153
:101190006E616C323C2F703E202020203C2F746406
:1011A0003E0D0A3C74643E3C7020616C69676E3D84
:1011B0002263656E746572223E3C2F703E3C696D01
:1011C00067207372633D2262616C6B652E6769668E
:1011D000222077696474683D2220255641403032D0
:1011E000226865696768743D223130223E3C2F7465
:1011F000643E0D0A3C74643E3C7020616C69676E0D
:101200003D2263656E746572223E25564140303240
:101210003C2F703E3C2F74643E0D0A3C2F74723E8E
:101220000D0A3C74723E0D0A3C74643E3C702061B1
:101230006C69676E3D2263656E746572223E41443F
:101240002D4B616E616C333C2F703E202020203C82
:101250002F74643E0D0A3C74643E3C7020616C69DE
:10126000676E3D2263656E746572223E3C2F703E50
:101270003C696D67207372633D2262616C6B652E01
:10128000676966222077696474683D22202556418B
:10129000403032226865696768743D223130223EF1
:1012A0003C2F74643E0D0A3C74643E3C7020616CBB
:1012B00069676E3D2263656E746572223E255641F4
:1012C0004030323C2F703E3C2F74643E0D0A3C2F60
:1012D00074723E0D0A3C2F7461626C653E0D0A3CCF
:1012E00042523E3C42523E203C7020616C69676E27
:1012F0003D226C656674223E203C68323E3C2F687D
:10130000323E3C42523E0D0A3C703E3C61206872C7
:1013100065663D225374617475732E68746D223E48
:101320005374617475733C2F613E3C2F703E3C4298
:10133000523E0D0A3C42523E3C42523E203C7020FE
:10134000616C69676E3D226C656674223E203C6864
:10135000323E3C2F68323E3C42523E0D0A3C7020E9
:10136000616C69676E3D226C656674223E556C72D5
:101370006963682052616469672032303037203CED
:1013800042523E3C42523E3C2F703E0D0A3C702081
:10139000616C69676E3D226C656674223E4B7572A6
:1013A00074205069657065722032303038203C42BC
:1013B000523E3C42523E3C2F703E0D0A3C2F626F23
:1013C00064793E3C2F68746D6C3E0D0A0D0A3C70CA
:1013D0003E416E70617373756E6720696E20417255
:1013E000626569743A3C2F703E3C42523E3C425228
:1013F0003E0D0A25454E44003C626C6F636B71756F
:101400006F74653E0D0A3C626C6F636B71756F742F
:10141000653E0D0A3C626C6F636B71756F74653E5F
:101420000D0A3C626F64793E3C64697620616C69A8
:10143000676E3D2263656E746572223E0D0A3C68DC
:10144000313E53746174757320506167653C2F6839
:10145000313E0D0A3C2F6469763E3C42523E0D0AF5
:101460003C6469763E436F6D70696C696572742087
:10147000616D205365702032352032303038207550
:101480006D2032333A35353A35303C76723E204362
:101490006F6D70696C69657274206D697420474363
:1014A000432056657273696F6E20342E322E3220BF
:1014B0002857696E4156522032303037313232313E
:1014C000293C2F6469763E0D0A3C6469763E42658C
:1014D00073756368657220736569742053746172F3
:1014E00074206465732057656273657276657273E4
:1014F0002028255641403039293C2F6469763E0D1D
:101500000A3C42523E3C42523E203C7020616C6993
:10151000676E3D226C656674223E203C68323E3C1C
:101520002F68323E3C42523E0D0A3C703E3C6120E8
:10153000687265663D22696E6465782E68746D22F6
:101540003E486175707473656974653C2F613E3CFB
:101550002F703E3C42523E0D0A3C42523E3C4252AB
:101560003E3C7020616C69676E3D226C656674223A
:101570003E203C68323E3C2F68323E3C42523E0D9B
:101580000A3C703E3C6120687265663D2268747456
:10159000703A2F2F7777772E756C72696368726156
:1015A0006469672E6465223E7777772E756C726961
:1015B000636872616469672E64653C62723E0D0AFD
:1015C0003C2F613E3C62723E416E70617373756E7A
:1015D0006720506F6C6C696E20426F6172642041AD
:1015E00056522D4E45542D494F20766F6E204B7527
:1015F0007274205069657065722031382E30392E32
:10160000323030383C2F703E3C42523E3C2F736D9E
:10161000616C6C3E0D0A3C2F626F64793E3C2F6812
:10162000746D6C3E0D0A25454E44004749463839D5
:101630006111001100A53F004D4D4D50504F5454C5
:1016400054416A445C5C5C3F73426262626A6B6BE9
:1016500016A71E6F6F6F5F7A6019AD211CB22556F9
:1016600094597B7B7B1ABD2323BA2C1BC325838310
:10167000831CCA267C8B7D1CD3268B8B8B2DCC3672
:101680001CD8261DDF289091911DE1281EE22921FA
:10169000E22C35DB3F2EE4389C9D9D3EE64740E63C
:1016A00049A5A5A547E75050E458A9A9A94EE85671
:1016B000AEAEADAFB0AFB0B0B064E66BB4B4B5B879
:1016C000B8B96CEC7377ED7DBFC0BFC0C0C0C2C2FB
:1016D000C2A6DAA9C9C8C993F198CCCCCCD1D1D1D2
:1016E000A5F3A9D5D5D5DEDEDEE0E0E0C5F7C8E795
:1016F000E7E7EFEFEFFFFFFF21F904010A003F00EA
:101700002C00000000110011000006EDC09F50D811
:10171000CBC954A9966DC8FCF974371A8C65026957
:1017200040B4A66FA72B2D10E0C545E2680D7DBB28
:101730001923E2097D3295C7A2918009753AC6C581
:10174000F5729D3E1B15130B09123F3D371E112BE1
:101750003538352E221D1B180F10062C39340B1E60
:101760002F383C382F241D1B1B150B061632300852
:10177000212E3538352E221CA4180804072A2C08DF
:101780001F272E2F2E271FA41B1908040229260805
:10179000191F2224221FC41B190802062D200B1812
:1017A0001B1DDED31B150B0212361A100FE0D311CE
:1017B0001000283F20140B13EA1B130B03094234BB
:1017C0000E0D0B0F18326CC880E1C1820200580C5C
:1017D00069914001840560102C601000C008263F0C
:1017E0006248306080000101020024608171080BB2
:1017F0000B0704189080026310003B25454E4447B8
:10180000494638396111001100A53F004D4D4D503A
:1018100050505252525454545756575A5A595D5D6B
:101820005D5E5D5D5E5E5E606060626262636363BA
:101830006464646565656969696E6E6E7070707701
:1018400077777878787A7A7A7B7B7B7E7E7E7F7FEB
:101850007F8080808181818383838787878989894D
:101860008B8B8B8E8E8E9091919191929393939777
:1018700097979A9A9A9C9C9CA5A5A5A9A9A9ABAB58
:10188000ABACACACAEAEADAFAFAFAFB0AFB0B0B075
:10189000B2B2B2B4B4B4B4B4B5B5B5B5B8B8B9BFF2
:1018A000C0BFBFC0C0C0C0C0C2C2C2C8C8C8C9C90A
:1018B000C9CCCCCCD1D1D1D5D5D5DDDDDDDEDFDED7
:1018C000E0E0E0E7E7E7EFEFEFFFFFFF21F90401DA
:1018D0000A003F002C00000000110011000006EC7F
:1018E000C09F50D8CBD1562AD86DC8FCF976B85ACB
:1018F000EC551A7946B5A68FA713351006C442A336
:10190000A1C0863EDECC31E97C369509A41181C8A0
:10191000843B9DA373629D461B1616120C0F183F45
:101920003D381F13273437342720188210120A2E0F
:1019300039360D1D2C373B372C211982130A091C0F
:101940003431081F26343734272017821508070E34
:101950002B2F061B23272C27231B828206050329F6
:101960002508151B2021201BC3161508040C302345
:101970000B1316181918D116130A0219371E17104F
:10198000DFD1101500283F231A0D12E916120A01A3
:101990000F423514110C1013152C549800414101BD
:1019A000002D86C080F040820204061028781000C6
:1019B0000089263330284860A0000101001EB46869
:1019C00032C405070703186440D12408003B2545AD
:1019D0004E4447494638396102000A00A20000A27D
:1019E000A5ED848FE5667CDD4960D62144DAFE01F1
:1019F0000200000000000021F90405140005002C7D
:101A00000000000002000A0000030A48342312010B
:101A100048001D5309003B25454E44474946383987
:101A2000615A005C00F700006C6E64BCBA4CB7B53C
:101A3000AC6161AF908CA8DADCAF6F66D8DCDE7188
:101A4000DEDEE28F8DD7DCDE88B6B6E07979D8F0BD
:101A5000F0B0EFF0878378A9F6F4E18C8E549F9F65
:101A6000DAA1A2A9C9C9E07F78F0EFF0C7E9F2A234
:101A7000BAB782C9CAB07878C1E9F1627569F192E2
:101A80009279EBF1FBC4C981918EEFF0F2708C8CEE
:101A9000C0DEDEFAE3E0C8B7B4FA8A84D7C8C9FB6F
:101AA000F8FD88A4A2787168BFA3A0F09F9FC077BB
:101AB0006E97FAFDB0DFDF9F8883C0BAB8C787840E
:101AC000F0FAFDC8F9FD717870D8CEC9C57F78E409
:101AD0008183A9D7E7FCF8FDA0B4B4979C98D8FC03
:101AE000FDE0FCFEFB9897C19793917770C08C80C6
:101AF00088DEE8AFE6EA87EEEF947270EEF0F0BCB5
:101B00007E78CC8178FCB0ACF2F2F3D4BFC89F9958
:101B100098F0C0C0FBD2D4FBA09AA8BFBFE0857BE1
:101B2000D9D1D3E1D3D3B0B1ACA6DEE8C9A8ACC05B
:101B300081809A7E79B4F7F39EC7C771C1C0B1EABC
:101B4000F07C7264E4EAE9DFA090D6F4F6B0ACACC5
:101B5000D8F8FD94C4C2C9D5DB94F4F688F2F0EC51
:101B6000F5F6C7857CC1F6FE5BF7F4FBF9FD7C78E2
:101B700070E4A19C93827EF1878BCCEDE0FCA6A45F
:101B80008EBCC09A7871CC7870FC8D8CE4A7A34F82
:101B9000928FFCBEBAFAFAFDBCEAE8FBD4D5997282
:101BA0006CA7928EB4DCDEBCB9B7EC897F61B7B6A6
:101BB000699A9461A1A06C847E7CE1E76780788853
:101BC000C4C27CA19B79D4D480CFD6C9EBE8A0C095
:101BD000C064D4CA97ACAE78A9A3E49A9EB4C5C732
:101BE000EC6967CC888898CCCE647E7799949A44C7
:101BF000AAAA92848769E8E9BCDFE8949497B4D7ED
:101C0000D5ECD4D4BCE6E8D4B9B5BCE0E17CE1E0E5
:101C1000ECB4B58C999284C6C78CDEE0D4A5A2FC46
:101C2000A4A0CCB2B4D4CECCD4746CB47C66B4C80A
:101C3000BAE0AEA4AACCCEBCF7F5647469FCD5CDED
:101C4000FBB4B8A492939C90926CD0CCA48B888B5C
:101C5000ACAA688583E48D85CCFBFDD48483B49ADB
:101C600098CCA098FCA9ABCCC2C0D49A9B9CC4C20F
:101C7000A4BCB674888878E9E294968ECC7668CC59
:101C80007C7274A2A5848A83FC9A99E4FCFEECEE33
:101C9000E7B27D70F1AEABFCDDD5FBBCC2ECE0D2AF
:101CA000E0B4ADB4EDE9C8C1C0BCB4AEE4F8FE64C4
:101CB000D0D6A4E9EA749C9A84988999BFBAB1965F
:101CC00092A6E4E2B0736AD9867EA9A2A6D9CCCE48
:101CD000E49A92C4AEA6F2A9A6BCD4CECCC4C28C5F
:101CE000DCD6D4B4B65CECE8ECA4A29C88806CC2D0
:101CF000C174AFAA84C8CF74ACAE9CDCCAEC817E40
:101D0000E4F4F694F0F6BC7E7ECC807EFC847EB457
:101D1000F3F67C716AE4F6F6ECA8A6B4D4CE8CADEA
:101D2000A6CCC0BAD47572B421F9040100003E00FB
:101D30002C000000005A005C000708FF007D081C12
:101D400048B0A0C18306990D5C23B0874385041970
:101D5000AE99280B818F893E98415008D1C71984CC
:101D600020438A1C499059C78110F45D6468704F04
:101D70009E2917053263699026C99B3849DA5CC8E9
:101D8000334F02311E640ADC3934A7D1A3327B9C65
:101D9000DC13D487CA811013D01121F0E91E590435
:101DA000F51145CA35A4C35D457DF498B1AB075420
:101DB0008852BE99A8EA23C732255DE3E264C8AC25
:101DC0004759851E58A2315BD28707791540105CB0
:101DD00040E719C69872131FFC0AF6E2293B3C50F3
:101DE0008993B8C624B31315EA34699A83478D12D0
:101DF0002CF7C0548CF464C4B1652FAE08626745FB
:101E00009A2C4EF6C464A66F81110E76827A50C267
:101E1000E086E18B14406D253DD2724166F41A8054
:101E2000DDAD01CEC072FF4A0CECB1265ABE0A3CB1
:101E30000682B8C1E0772B2C4F881BFFAD5B376360
:101E4000C9192ECC3E31B142B6873D0B74A5B129DC
:101E5000AE420D316B3C3C69D3E6D49E35B28880EE
:101E6000C308C3155460570E2548D0582EA0E1432F
:101E70001C48E41187122728214510CB1CE6832833
:101E80000968308240B2DC20C3877BF0008E353C8D
:101E90008957DC2E6529B5E00C17D0C3CC1E69C864
:101EA000B20718300491862EE3D0D4C317E1F8119D
:101EB000D41A4E7CE3CB19D5C12002348845A4E264
:101EC000627691E5504C63E990DE1EABE8C21028C3
:101ED000C4B841411C03E933033D36C430543C606F
:101EE000800901163800729386C431B3CB9833B899
:101EF00028931EF3E8408F073FA4F1833ABBA081EB
:101F0000060419CDC44C183A58F189427B8892CA0C
:101F10001A165041C9024D0DE541A561A9C890436B
:101F2000338C999A4C33E880820E3DC4C1431AC069
:101F30004030831E2D2AA4CF1863A4FFB750650D2F
:101F40000C218AA598FA55D4813941245146ABBA5F
:101F5000A0C70C103183DE1866CCE0C31EF5F0225A
:101F6000CD11174849E82E28D0A083B2027D21E781
:101F7000108DC926D01339E440C12FBDF4C2030F20
:101F8000BD5C615193999664D2AC16B8B806394AD3
:101F9000045565AC4B141A2A0D28C83A8209E0147E
:101FA000E042034A39A4070DD62ACB123DBB589014
:101FB0005F1C259C22317770F4D15B0D0CC8A30403
:101FC00034BCAE28680F1E98C0801D3988A5033E1A
:101FD00063EC62590F7AB04143B217359106299DDF
:101FE00082A5EA186CB0A103A1138922001731FC65
:101FF000F28F09264C22C3370C9450C209CF54F0FB
:102000008D0C4E5CAA580F0D5CEB81060C7CD3C482
:1020100008CC1C8C8FAC02517B0D1B2E2C6B822E9E
:102020009490D080B210B8D005D910AC7142097626
:1020300048B10AD12A301084040BE4FFD0D4A5CBD8
:10204000A85542AE0799966243C6C62A0E126F9CE7
:10205000C2C00AA2F4A0030DD152596DBF0A2DD3FC
:1020600007283D84A18749A136E3890826B4E1B455
:102070000C7420D1440923EC51B24039C094870636
:10208000CB3CD1B152A60D176A18BF30D01D080C39
:10209000244006A26390AA500FF3B08142315FDC66
:1020A0008805362E44BB0B04E8B8E2471AC754E053
:1020B000CC1B5238E137EC3E4800480E4FA4E28476
:1020C000133780F0A179ECCBD5353DCBBC914B13C8
:1020D00032DC50030CD534836C1875CE30060A5DA3
:1020E000400437F6D18D4510010544A859144C50D1
:1020F000030EA44F162CA9140B725002068840043C
:102100004E3881330CE08486E00E2A24E108423CFC
:10211000E08B249CC00E46A8431D9C218569940138
:1021200005A35A153EF0318F0FECE0159A70010AA5
:10213000CCB00917B8C00ABAF00207FF7C211B8691
:10214000E8431F66094A0264E08B4904C109D05084
:10215000C61BF24014111AEE2C09220FFB1842C2C2
:102160005878C00E78C88C116A008E0FC090063E59
:10217000C407D91AD00017E8A00B3A48473A7C4860
:10218000050D702009CF48CABBF471821C38C10804
:102190004678437B4E61249A20D124FAD848FB0A22
:1021A000E710342CA14553AA8C0F40F0060F8CE0A9
:1021B00014F270021DE8F08B4DD04079FCD2C118AA
:1021C0000E88337E61821D17B8800BB800831ADC3D
:1021D000200F4E2148504EA18CA6C923014F38052F
:1021E00012A4B0873D40A0609DFAE0BB425297B177
:1021F00058A0667799513D6490836738E10927A814
:1022000007039E300314E42C673BC4070CABA50006
:1022100062D8005A17988506267183A80D44141EAB
:10222000F8452F39500723C0E109B2C08306FE8369
:1022300080638E490F7AC0DD1511C2FF297A84C1EF
:1022400005C1F481246AF006273C4362807186123E
:10225000D0300684CD430B08DBA116D6F68817ECE8
:10226000E20FC9B80015606084249CE2757CF2011D
:102270002A24F0846FDC4005E1F041050C009A4E01
:102280004C010D7AB88095EAB44F84D08541FF0C9B
:10229000C31198010D5DD0216B1500242041A08F42
:1022A00022204C0B3A80C53568100A0C4060097C2E
:1022B0002880373A90810B58A11E4988453EA221BB
:1022C000100FF0C2032718800C2A90490F38A10282
:1022D000F618C11780F08919144158F9ACE915E9CD
:1022E0005297198421A716A806277E00877A806056
:1022F000121DB5C70022514D7EB141A9D918063231
:1023000040A1CA5700A103FFB4422E62118B6FFC9B
:102310004257E1585A1B9CD1CE117800063738C578
:1023200008124108CF5DA02C1DF30AA766508CB798
:1023300036205FAAE0C50A72D90606FF2C030710F3
:102340006828C23E890205B8410E79AAC2213431FB
:10235000042B4C401EECAC000C9A72821AE0C11E99
:1023600049E0802C7290877A482007EA08C40588E3
:10237000C02ABEA4762454D321BF66600A4E68A04A
:102380008F1319411052310F84B94C793CDC040A87
:102390002E0000282CE1132C18400DEC710A0ED0F1
:1023A00001126D194103EB908F53E8E71B1A30853A
:1023B00005B4318B19348050486457086B22161DC0
:1023C00062530F8BE0453D1200030D98E0061A6042
:1023D000C419D9900D0530620C2140812232200AA7
:1023E00004104003F2E0C113F670472910C8072516
:1023F000AC03123C9003112001104B284532D04011
:102400000F6C39A95735A98B1E44F93F2DB0E01F39
:10241000E7BA813D8CA0014FBCB1A10AB8051044B8
:10242000E5802D14000109C81A0FFC068D3A70A032
:102430000DCBC8CB08DEF08D1FF8E0FF0470C08222
:102440003E10108C3FCCC92CBFC249311364A70584
:10245000A1210C0D1DC33460008D11E4E1191C6035
:10246000802B8E8033366C421B6E38990EF8408D6F
:102470006EBCA10E99F44B7F2B5081492C43202731
:1024800074C21A4E918639D0830C31F8E5948E636C
:102490009961F2A4AE7AF0215C83C9978CF44087ED
:1024A00045B00001E8600006C8C00B37B00409C69B
:1024B000B0011816A108CA23822658A0012F544043
:1024C000064D0141054EF10C6518E1097939C11E2F
:1024D000E220054BC8940B7160096382256B80B6BE
:1024E000C8206389B50ED66D251F0EEB21554241DC
:1024F00018D001C65334C117CAD0001926B7CD6A07
:102500008D610813F8C70D8C70837AC4049379F039
:10251000C029BC00870F11A90248E8861B4950A8B2
:1025200039A14754302CDE4C550692BAA247A6FF7B
:10253000DBA6B004E5C644D5A30227FF78422E836C
:10254000E0075B880A61D7404103409185493841E3
:10255000060C90004656C0809239C10E0380830459
:102560004E504229B4020DE6466AC8ADC9AF7ED1CD
:102570009AD58BD9C592FFE7B25115001455A042E8
:1025800018A24501248416786F5041303491BC4F15
:1025900086210322C80533E9D07096F080013E7091
:1025A000020372210F0D489303F908823AF4F056A2
:1025B0002DB82CA219B792CA3A7298621A2E4A3EC6
:1025C000FCDF2640A18B6F1800061318C20F832171
:1025D00082139CC009A778830940D1003398A101D8
:1025E00036C0813C7A7E02242460220A69420DF2C0
:1025F000F086DB1881013078C06B80800614149B54
:10260000E963D31304549D90E9107E2837ED143EFE
:102610003310440766E1161D903C1370B08CF3D95B
:10262000A30EDF78C092B5400254E4CD0E3EC883BD
:102630006D87F46623B4C108CA504BFF34CEF00551
:102640002E246214465543D361A8837C1EB9F71427
:10265000B609441620056704211243D8042632E146
:10266000823088E00D356004B1500715D00247A0D4
:1026700005CD0005AEF44E60953ECB22104E900481
:10268000AFA7019CC0046E842C3B84026AA07E6CC0
:10269000300F00056FB5761C8B444C5D550206F07B
:1026A0000DD6F00963D00505900CC5C30274905C8B
:1026B0003710045070042E20000FE034BC5032CF8D
:1026C000504E2C8119CE20031A100956E002A32483
:1026D0004A0E400465C70663D05D26611721781352
:1026E0004F982065911A392005747002CCE0467A23
:1026F000B00528300F5490061CC001414000C1E0D5
:10270000096130042C10806D700502110DF2101E4D
:102710006F960B8EA701FE600143300416F005583A
:10272000070F5530072FB06E71C567C8944507B1C4
:102730002951126BB2166BEFA60F3FFFF00051B09C
:10274000062C430F170043178009C6B00AAEC00419
:10275000477057F0500FCEC600921014271004E1B6
:10276000B1070C940B300004BB30048E300BDB60DF
:10277000092D000531C00D3B800165E04364116BFC
:10278000E4D66E35232FB36117890743D884021A24
:10279000F70EF8C404B4800355F00AD4400F666005
:1027A0004DD970017AA0050EE0437F4000FBF50C87
:1027B0000CB03EE2304F7B400E6D703F36A00532CC
:1027C0004702F1D00FD2F04B431053EDD0083094B4
:1027D0000DDB244AD6D46F822825FAB032735272A8
:1027E000FF1372B0320FEFF05668A00A62300D503E
:1027F000E006EE200821C0064B055F0E400F570093
:102800006398D70403E10162C0340C300926300D0F
:10281000618002D7D00829B00DDB9008114008185C
:10282000F00276150A34700D631351F3308FC5E34F
:102830006E75A24FC621131EA76E2EFF300A5C9044
:1028400001243002D0B007E880005C700EEFB05B6E
:10285000ECE702549091E190030C700A2BE1032302
:102860006007DC0103557004F3A05421100A8E8028
:102870000D0AA0003B0004B7500DD41006111572CC
:10288000EBE643107006595430E4D167ECB25ABB02
:102890007006E8000485200442C00EB5707E0DA0CD
:1028A00000D5E232D9E00068400937F0067EA30186
:1028B00025E02D130102CEA00B643004A2F25E28A5
:1028C000E000A23206D4B00722F000AEA009FFA3B8
:1028D000038C6025C35227BC225785D23EC6B26402
:1028E0003A009007B04D1BA8063A600A41C0001D8F
:1028F000541D2B401388760CADD000F3C808C5A03A
:1029000003D10843F300013EF5005CB02AB4D66A57
:10291000BB7214EF328573827128803263E0005AF3
:1029200080622BA903A8603F9EE503D6600D2CC1F1
:102930006D521009D4A0038610023AFFD00083F034
:1029400008805609A1E002CDC00537E00CBC500D4F
:102950009AF04F52929C6FF27E62217C53C7749F13
:1029600094624470572FB00548450541E00C6B4117
:102970008A127011710003588009F255049770078C
:102980007C70048330086C94026E200D68E20C1C8D
:10299000000E5CC09C1BD767FB04273E122CB07254
:1029A000462C09780170070DE008B540089A8006AA
:1029B000FBC01F70311080C0102BC00B3BA0030C5C
:1029C000D95B0DA009D4400888E0438F2004E0F0D3
:1029D00000AC700C11870D2FD7749E39937CE66A7A
:1029E00006D210AB428F7F8730AB39365FD8088272
:1029F000300354C00E29000114900653664E7EF138
:102A000003790009BA400B461502C56606E71008AF
:102A100019D0000E608C45700EA42004DB0004F079
:102A2000C007A2C45BD79471C2F28B0F512C1091D6
:102A300048108074F4684DD854A5CAFF13995AC041
:102A40000F2F600119400567300E41E00B20E02692
:102A50000371025260027EB0049713029FC40818EB
:102A600050008CC090A1D400CDA009C5109DA262D9
:102A7000064B578CC5430F45B61753723C63D1299B
:102A8000E5B6AB8AB86EB1F272A3D20E83D05A68A3
:102A900060030F009B4A900A04610D52A002E558A2
:102AA0002D9FE45E29664DD7A07E19D76FB10250E5
:102AB000FF5472ED065045466B2E524CF8F9992C96
:102AC000C26751122CD06A060AA0085F3803B7709B
:102AD0000F69160D5130246B900548D00A33E00081
:102AE0002E93628CBA5BBBF57763A33C33451664C7
:102AF000C122065BB0E69A104FFA7B95A12AB8E98D
:102B00005E9F045FD4700830F03D94E21769D007EF
:102B100050F0078F3943A5C4061BA04DD0BAA811A9
:102B2000BB4DB1029AC168AE1F849C76C1502ED3B2
:102B3000922B490363400204F00F39FFC010CAFA18
:102B4000044D8004E390018FA93C0E100AF2583C1A
:102B5000C852A5C49833FECA842E901A2C411EFB7D
:102B600014852171713BE45EDBB4545DC005FFE068
:102B7000210201087B700A35F00F0250890EB90559
:102B8000ED503C8C60016DB492277A4D55BA54A13A
:102B9000542720444C35251675B5A48D8A02483536
:102BA0008FA2D0071A400E7E210BA7500174D00FC0
:102BB0009FA007DB64065AF0018158068990080936
:102BC0001902D5EAB68ADAA848FBB66E591A0CB2D1
:102BD000A4F3286BBC399E9E200A0F1004BAF01F84
:102BE0007B6007410003A6600547D0005A50045A95
:102BF00060577A500A836092C3700707B00192DB76
:102C0000A89EE943C4382A7AC0335CC12916C6A4F9
:102C100032397563400FD360090B800A22A001ABE3
:102C2000A00141A00238A00A56300A1D8009A580E3
:102C30000B811008C26001B630079BFFC03F61A046
:102C400008FA1AADEE355376B164EC17060C73B979
:102C500022713CFBE8ABED370384A264938346C446
:102C6000A7020970023F000641500352A00BB33087
:102C700004D8200758D00DD5800E364000592006C4
:102C80008E3906F3D000D4E008CDB0A41B38364B03
:102C9000CB1173D2AB9BE9BE08611273B2BA9EF33B
:102CA0006E3121893A34364370080C600F93F04E30
:102CB00015A20B3C0004BB790168F00A584009A238
:102CC0007006E5800441500D4790873B2007B340D4
:102CD00005CD608E6A6BADEE371D240A43BB908F25
:102CE000245817BBF04890F47BB7467544C009746C
:102CF000900449307AB9500271200D4BF0B03B740A
:102D0000019E6009FD6001DE700F35600212000354
:102D10008700045CE006A4B0036E554A1C182B8D96
:102D2000216E1627252B0B25097B129BA2075437F2
:102D30000647700FD3366568C5002DFF400AC530C1
:102D400006864003EAF76F58E00F5A500C5870316E
:102D50003040069F8006474005A3700E6DF49C8AA4
:102D60006A8C60831805934573FB84E56138C7520C
:102D7000752E500DB081076F9004D0170462500D6E
:102D80007C29AA6AC00666500642600EF3500450C1
:102D90009005FFE007737001FDA8030A800B5AF04D
:102DA000BA52AB3C275B388637B72004A515D697B7
:102DB000A3A20F50100E7B40076F606D82F404AE2B
:102DC00020B44C47625B900C9A39067F300DD3409B
:102DD000022EC0061BB801C5B305F3300F058B1ECC
:102DE000C488C7B36293D40C5E868B304DD8037B06
:102DF00000035310050C800778C000F51007E18030
:102E00000C5A20B208830F26265EEB8628D5B281A5
:102E100056A20507E4BB4AB10B1606430055385CC1
:102E2000C1112CF39801BD06D010046B100CBAF040
:102E30000CCFA0017DF0040450053AFF340F63006D
:102E40000B4C5A76FCF23FB8AB7E0055350B392A55
:102E5000322175186725501B17753BB0D4B1072573
:102E600000061E700B38E0044AF00F22E00F4250BB
:102E70000045102B7E8730B06A06FE6A25D08A0294
:102E8000ACE2D1A23A2AB596B9BE4B2C89F1848125
:102E9000B26E1C87A084260A9680034F1004F5802A
:102EA00003E610A76EE44366507579E29166E74643
:102EB00039830F5A501668A0A321902CBEE2031E3E
:102EC0002D4AD7E2C146E1104B80063339147130E8
:102ED0000ED3F005CCD60B2340079B470265F05676
:102EE000FCA343F8C02FBC0BD033B0042EE0D54C6C
:102EF0003893539727D8C21252D77FAC62CD91FD39
:102F000015054328F00109FD00018BE061DA660038
:102F100074E00A0D60D3816A8455D729A584027BA9
:102F200081061025B371B59C9D9BC752FA745D3123
:102F3000850F211067200E9DC01423FFF003C740AA
:102F4000447150034850051DD9842CA20766A04641
:102F50003AF048EFBC546160302E132B4A81444B49
:102F6000A63CA55C104784D4D3FC141731243C90B4
:102F700037A2164D3FC0B13034938006D24A71C299
:102F800068548538D32F8DC1D83A1443DE15A52A4D
:102F9000E2DF1E000874200527B00623600C3FF016
:102FA00005466806C6C332FF330F71E53F9F941E86
:102FB000C2588F46662C46A805DD75384F42107BF7
:102FC0004001F780041DC4D4E1800EBBA0039239F8
:102FD00088D5E474A06361B262173A2AD61DC12075
:102FE0006D04B7351E165293037E000E38D0E11ED5
:102FF000D0099D90119D778D8337163014062AD302
:10300000E2017D1163012BA59C2074F2D671AB22E5
:103010001E200B7E80050B00271040D4F6DC03F940
:1030200058C5CC7DCAFE43DF54B2D7114ED26810CA
:103030002FF087143671184FC00238FFC00253C0FA
:10304000109D10034C026BFC03152C332A83072CB4
:10305000A252CA30CE3F7866933DB07B471D17130E
:10306000C1457BF0043F4000E2D055CBC23119315D
:10307000279A3E1B52573CB55617BC59DBC1372C1B
:103080006ACE11B4F1E43ED009E56009BF603B9817
:10309000E2236301E6676DE2F9FDE3FAACC445069D
:1030A000A28562DB5DF1117EA10AC0002636E1DF58
:1030B000436130C3A2107441D4F97D6BEDA7147A3B
:1030C0001C4C27D1CF5D51E8FF2D132AC11248B403
:1030D0000BCBAEEDB6C68827C1321FB820B91AE1B6
:1030E000BADE2487E12D625138BB70049F226EC482
:1030F000198230AED6297B17F70E12F25738AAB2D2
:103100006A4941D94636D468A0323481DD078FD46C
:103110000A5210B91A8575A548F4CEF0153FD27E33
:103120000CB586C86ACEFEF17171F1186F12DF65B9
:10313000F289E1F1EE52F22CAF222E07DF17E4AE56
:10314000180101003B25454E44485454502F312E60
:10315000302032303020446F63756D656E742066A8
:103160006F6C6C6F77730D0A5365727665723A20D7
:103170004156525F536D616C6C5F57656273657247
:103180007665720D0A436F6E74656E742D54797096
:10319000653A20746578742F68746D6C0D0A0D0A99
:1031A00000485454502F312E302032303020446F9C
:1031B00063756D656E7420666F6C6C6F77730D0A46
:1031C0005365727665723A204156525F536D616C59
:1031D0006C5F5765627365727665720D0A436F6E38
:1031E00074656E742D547970653A20696D616765F8
:1031F0002F6A70670D0A0D0A00485454502F312E63
:10320000302034303120556E617574686F72697A80
:1032100065640D0A5365727665723A204156525FB5
:10322000536D616C6C5F5765627365727665720D84
:103230000A5757572D41757468656E7469636174D8
:10324000653A204261736963207265616C6D3D224D
:103250004E65656450617373776F7264220D0A4323
:103260006F6E74656E742D547970653A207465784C
:10327000742F68746D6C0D0A0D0A003430312055BE
:103280006E617574686F72697A656425454E440095
:103290006C65646F66662E676966006C65646F6E48
:1032A0002E676966000000636865636B65640050A3
:1032B0004F53540053746172742054656C6E65747E
:1032C000205365727665723A0D0A00D9000AFA0039
:1032D00000000000010400000000000000000000E9
:1032E00000000000000000000000000000000000DE
:1032F000000000C7D6AC720800000025454E440A05
:103300000D4E54502054494D453A202532693A25F6
:1033100032693A2532690D0A002A2A204E5450207B
:10332000444154412047455421202A2A0D0A004B8C
:1033300065696E204E545020536572766572206721
:103340006566756E64656E21210D0A002A2A204E7D
:103350005450205265717565737420676573656E8E
:1033600064657421202A2A0D0A002A2A204C43442D
:103370002044415441204745542042797465733AB2
:10338000202569202A2A0D0A00474554202F676C02
:103390006F62616C776561746865722E61736D78B8
:1033A0002F476574576561746865723F4369747926
:1033B0004E616D653D5061646572626F726E264349
:1033C0006F756E7472794E616D653D4765726D61A2
:1033D0006E7920485454502F312E310D0A486F73A6
:1033E000743A207777772E776562736572766963B2
:1033F00065782E6E65740D0A4B6565702D416C699C
:1034000076653A203330300D0A436F6E6E65637413
:10341000696F6E3A204B6565702D416C6976650D5C
:103420000A0D0A000D0A0D0A0D0A446174656E202A
:10343000416E666F726465726E0D0A0054435020CF
:1034400045696E7472616720676566756E64656E46
:103450002028485454505F434C49454E5429210D6F
:103460000A005443502045696E74726167206E698A
:1034700063687420676566756E64656E20284854BD
:1034800054505F434C49454E5429210D0A00415286
:103490005020526571756573740A0D002563000034
:1034A00011241FBECFE5D8E0DEBFCDBF11E0A0E6FE
:1034B000B0E0E8EEF7E702C005900D92AA39B10737
:1034C000D9F715E0AAE9B1E001C01D92AE3CB10701
:1034D000E1F70E946F1A0C94F33B0C940000CF921A
:1034E000DF92EF92FF920F931F93CF93DF938FEFB3
:1034F0008ABB84BB81BB60E875E280E090E00E94FB
:10350000F61A88EC90E09F938F930E94B41B80EA98
:1035100090E09F938F930E94B41B8BE690E09F9363
:103520008F930E94B41B80E090E0A0E0B0E02DB744
:103530003EB72A5F3F4F0FB6F8943EBF0FBE2DBF78
:1035400000000196A11DB11D803432E493073FE0D5
:10355000A30730E0B307A1F70E947F280E941D3522
:103560000E9470368BB780628BBF78940E94873739
:103570000E94313798E6C92E90E0D92E8FEFE82EC1
:1035800084E0F82E04E510E0CEE5D0E00E94862726
:103590008091750480FF19C0DF92CF920E94B41B06
:1035A000C7010E94832D0F900F90882319F0DF939D
:1035B000CF9302C01F930F930E94B41B0F900F90E4
:1035C000809175048E7F809375048091980190910D
:1035D0009901892B41F484E794E0909399018093B9
:1035E00098010E9431370E942A35D0CF9B01AC014F
:1035F00088E98AB984E0220F331F441F551F8A953A
:10360000D1F760E074E284EF90E00E94483B2150E3
:1036100029B9809175048B7F809375040895982F44
:103620008091750482FD03C05D9BFECF9CB9089517
:10363000CF93DF93EC0103C021960E940F1B88817A
:103640008823D1F7DF91CF9108951F920F920FB683
:103650000F9211241F932F933F934F935F936F9378
:103660007F938F939F93AF93BF93EF93FF9380913B
:10367000750482FD4BC01CB1812F0E940F1B8091ED
:10368000750480FF04C080917504826028C01830E2
:1036900069F480919A0190919B01892B09F452C0A1
:1036A00080919A0190919B0101972BC01D30D1F41C
:1036B000E0919A01F0919B01E250FB4F80818C35A3
:1036C00089F0E0919A01F0919B01E150FB4F10824B
:1036D00010929B0110929A018091750481608093F1
:1036E000750430C080919A0190919B01C19750F56B
:1036F00080919A0190919B01FC01E150FB4F108356
:10370000019690939B0180939A011CC020916000C8
:1037100030916100809162009091630001972817B9
:10372000390781F08CB1F9018193F0936100E09346
:103730006000E053F54031F4205330403093610095
:1037400020936000FF91EF91BF91AF919F918F9176
:103750007F916F915F914F913F912F911F910F90AA
:103760000FBE0F901F9018959F92AF92BF92CF926D
:10377000DF92EF92FF920F931F93CF93DF93CDB71A
:10378000DEB766970FB6F894DEBF0FBECDBFFE0161
:10379000B496E190F190FA83E983992423E0A22E74
:1037A000B12CAC0EBD1E9DE0C92ED12CCC0EDD1E61
:1037B000F7018491882309F48AC00894E11CF11C64
:1037C000853209F081C0F7010894E11CF11C2491B5
:1037D000822F90E0C0970A9710F0822F0BC02D87A0
:1037E0001E86C6010E941C3A982EF7010894E11C1F
:1037F000F11C8491893661F18A3628F48236F1F021
:103800008336B1F61DC0833741F0883721F08F36FB
:1038100079F648E01EC040E11CC0E981FA81329689
:10382000FA83E9831291029104C00F5F1F4F0E9437
:103830000F1BF80180818823C1F7BACF42E009C08D
:10384000E981FA813296FA83E983329780813CC01C
:103850004AE0E981FA813296FA83E98350E0B501C2
:10386000929182910E94063B20E030E0F501E20F48
:10387000F31F80812F5F3F4F8823C1F721503040D5
:10388000892D90E028173907D4F4921AA0E0B0E00F
:10389000292D30E005C0EA0FFB1F80E380831196DD
:1038A000F601A217B307B9F7AC0DBD1D1C92B50107
:1038B000C6010E94D13AB601C5010E94DC3AC50199
:1038C0000E94181B992474CF0E940F1B71CF66961B
:1038D0000FB6F894DEBF0FBECDBFDF91CF911F9121
:1038E0000F91FF90EF90DF90CF90BF90AF909F909F
:1038F0000895CF92DF92EF92FF920F931F93CF9391
:10390000DF93CDB7DEB724970FB6F894DEBF0FBEB6
:10391000CDBF6C017A018B0120E030E0AE014F5F3A
:103920005F4FD601A20FB31F0E94723B802DFA0198
:10393000E20FF31F80832F5F3F4F2430310589F75B
:1039400069817A818B819C816F3F2FEF72072FEF06
:1039500082072FEF920711F4C801B70124960FB622
:10396000F894DEBF0FBECDBFDF91CF911F910F91B5
:10397000FF90EF90DF90CF90089520E030E0F901C4
:10398000EE0FFF1FE20FF31FEE0FFF1FEE0FFF1FE3
:10399000E65DFB4F82859385892B59F41082118255
:1039A0001282138214821582168217821086118663
:1039B00005C0828593850197938782872F5F3F4F4C
:1039C00025303105E1F60895DC0120E030E0422F9A
:1039D000E22FF0E02F5F3F4FEE0FFF1FEE0FFF1FB4
:1039E000E456FE4F80819181892B89F7453020F480
:1039F000B183A08373836283089540E050E0A42FD5
:103A0000E42FF0E0EE0FFF1FEE0FFF1FE456FE4F16
:103A1000208131812115310529F04F5F5F4F281733
:103A2000390769F7A53010F4718360830895DC01CC
:103A300020E030E0422FE22FF0E02F5F3F4FEE0F0B
:103A4000FF1FEE0FFF1FE055FE4F80819181892BF4
:103A500089F7453020F4B183A0837383628308958E
:103A60001F920F920FB60F9211248F9380916804CA
:103A70008160809368041092C6011092C701109271
:103A8000C8011092C9018BB78F7D8BBF8F910F90AA
:103A90000FBE0F901F901895CF93DF93C091DD015B
:103AA000D091DE0160E070E086E0C830D807C1F454
:103AB000FB01EE0FFF1FE60FF71FEE0FFF1FEE0FCC
:103AC000FF1FE65DFB4F2681378140855185809140
:103AD000ED019091EE01A091EF01B091F0011AC0BB
:103AE000C830D105E9F4FB01EE0FFF1FE60FF71F09
:103AF000EE0FFF1FEE0FFF1FE65DFB4F26813781A4
:103B0000408551858091EB019091EC01A091ED01F0
:103B1000B091EE01281739074A075B0709F45BC02B
:103B20006F5F7F4F6530710509F0BECF20E030E058
:103B3000F901EE0FFF1FE20FF31FEE0FFF1FEE0F55
:103B4000FF1FE65DFB4F86819781A085B1850097B9
:103B5000A105B10509F044C086E0C830D807D9F402
:103B60008091D70180838091D80181838091D90190
:103B700082838091DA0183838091DB018483809149
:103B8000DC0185838091ED019091EE01A091EF0120
:103B9000B091F0011CC0289749F58091D70180832E
:103BA0008091D80181838091D90182838091DA014B
:103BB00083838091DB0184838091DC018583809104
:103BC000EB019091EC01A091ED01B091EE018683A3
:103BD0009783A087B18784E690E09387828706C0A9
:103BE0002F5F3F4F2530310509F0A2CFDF91CF91F4
:103BF0000895AB01BC0180E090E09C01FC01EE0F58
:103C0000FF1FE80FF91FEE0FFF1FEE0FFF1FE65D0E
:103C1000FB4F86819781A085B18584179507A607FC
:103C2000B70739F0C90101968530910531F725E0D4
:103C300030E0C9010895CF93DF93EC01CB01BA01C5
:103C40000E94F91D853009F1DE0140E050E090E06E
:103C50009C01220F331F280F391F220F331F220F01
:103C6000331FF901E40FF51FE65DFB4F80818C9354
:103C7000FA01EF5CFA4F8081FD0186834F5F5F4F51
:103C800011964630510569F0ECCFA1E3B5E0FE0195
:103C90008FEF80838D918683319685E0A733B807B7
:103CA000B9F7DF91CF910895EF92FF920F931F9391
:103CB000FC0179018A0110C080812181329690E057
:103CC000982F8827820F911DA0E0B0E0E80EF91E22
:103CD0000A1F1B1F625070406230710568F7672B26
:103CE00051F0808190E0982F8827A0E0B0E0E80EA6
:103CF000F91E0A1F1B1F9801442755278FEF9FEFBE
:103D0000A0E0B0E0E822F9220A231B232E0D3F1D7C
:103D1000401F511FCA01AA27BB2740705070820F55
:103D2000931FA41FB51F809590951F910F91FF9031
:103D3000EF900895AF92BF92CF92DF92EF92FF92F1
:103D40000F931F937C015A016B010E941B1E88E098
:103D500090E0F701958784878701025F1F4F80E419
:103D600090E0F8019783868380E880878091C40182
:103D70009091C50101969093C5018093C401292FAC
:103D80003327982F8827280F391F3583248385E40C
:103D9000F7018687F8011182A08AB18AC28AD38A84
:103DA0008091690490916A04A0916B04B0916C04B5
:103DB00084879587A687B7871386128620E030E030
:103DC00040E050E064E170E0C8010E94541E292FD9
:103DD0003327982F8827280F391FF8013387228728
:103DE0001F910F91FF90EF90DF90CF90BF90AF9019
:103DF00008956F927F928F929F92AF92BF92CF92CF
:103E0000DF92EF92FF920F931F93CF93DF9312E213
:103E1000C12ED12CC80ED91EBC01625F7F4FEB01B1
:103E2000EC84FD840E851F8540E050E086E190E043
:103E3000489FF001499FF00D589FF00D1124EA585A
:103E4000FB4F80819181A281B3818E159F05A007D0
:103E5000B10709F0A0C024813581D6018D919C91D4
:103E60002817390709F097C0E60188859985AA8542
:103E7000BB8580879187A287B3878C819D81AE8126
:103E8000BF8184879587A687B7878D85808B838937
:103E90008F3F11F083E0838BEB018A819B81F82EA9
:103EA000EE24892F9927E80EF91E8CEE9FEFE80E7D
:103EB000F91EE6018C8590E0807F9070959587953E
:103EC00095958795E81AF90A00E010E0A484B58476
:103ED000C684D78424853585468557858485958510
:103EE000A685B78564847584868497842070307035
:103EF0005070232F342F452F5527AD2CBB24CC24B5
:103F0000DD242A0D3B1D4C1D5D1D8070A070B0701E
:103F1000BA2FA92F982F8827280F391F4A1F5B1FF8
:103F2000962C882477246624260D371D481D591D9C
:103F30002E0D3F1D401F511FE12CF12C1FEF012FB3
:103F4000112DE222F32204231523EF2CF02E012F52
:103F50001127852F9927AA27BB27E80EF91E0A1FCC
:103F60001B1FDA01C9018070A070B070BA2FA92F91
:103F7000982F8827E80EF91E0A1F1B1F522F44276F
:103F800033272227E20EF31E041F151FE486F58651
:103F9000068717874EC04F5F5F4F4530510509F0C8
:103FA00045CF20E030E086E190E0289FA001299FE6
:103FB000500D389F500D1124FA01EA58FB4F8081B3
:103FC0009181A281B3810097A105B10561F5E082DD
:103FD000F18202831383D6018D919C919583848312
:103FE000E6018A819B819783868388859985AA8546
:103FF000BB8580879187A287B3878C819D81AE81A5
:10400000BF8184879587A687B7878D85808B128A25
:10401000118A83E0838B148AFA01E557FB4F808174
:104020008E7F808306C02F5F3F4F2530310509F01A
:10403000BACFDF91CF911F910F91FF90EF90DF905A
:10404000CF90BF90AF909F908F907F906F9008958A
:10405000EF92FF920F931F937B018C0180E090E021
:104060009C0186E190E0289FF001299FF00D389F88
:10407000F00D1124EA58FB4F80819181A281B38118
:104080008E159F05A007B10729F4848195818417B7
:10409000950739F0C90101968530910509F725E0AA
:1040A00030E0C9011F910F91FF90EF90089560E0FB
:1040B00070E0E62FF0E0EE0FFF1FEE0FFF1FE05560
:1040C000FE4F4081518141155105A1F02091F5012C
:1040D0003091F6016F5F7F4F832F9927322F222770
:1040E000820F931F4817590721F70280F381E02DB3
:1040F00080E0099508951F93CF93DF93182F60E018
:1041000070E0282F30E086E190E0289FD001299FC1
:10411000B00D389FB00D1124AA58BB4FE62FF0E028
:10412000EE0FFF1FEE0FFF1FE456FE4F408151813F
:104130004115510581F0ED012E813F818E819F81D6
:104140006F5F7F4F892F9927322F2227820F931F6E
:104150004817590719F70280F381E02D812F09953F
:10416000DF91CF911F910895863038F5282F30E0E8
:1041700086E190E0289FD001299FB00D389FB00DB7
:104180001124FD01EA58FB4F108211821282138222
:104190001582148217821682108611861286138663
:1041A0001486158616861786108A128A118A138A33
:1041B000A557BB4F8C918E7F8C9308954F925F9241
:1041C0006F927F928F929F92AF92BF92CF92DF9227
:1041D000EF92FF920F931F93CF93DF932C0170E028
:1041E00086E190E0689FE001699FD00D789FD00D37
:1041F0001124CA58DB4F8E819F819093F4018093E4
:10420000F3018C819D819093F6018093F5011092CA
:1042100006021092050281E094EF909302028093CF
:10422000010280E58093FF01EC84FD840E851F85EB
:104230008C859D85AE85BF852C853D854E855F85AA
:10424000AC84BD84CE84DF8480709070B070692EA1
:104250007A2E8B2E9924E12EFF24002711276E0C35
:104260007F1C801E911E207040705070542F432F71
:10427000322F2227620E731E841E951EDA2CCC2448
:10428000BB24AA246A0C7B1C8C1C9D1C88898093EF
:104290000002888981FF17C00894611C711C811C71
:1042A000911C82E08093070284E08093080281E001
:1042B0008093090284EF80930A0280E68093FF01D5
:1042C000F4E04F2E512CA4019301207030705070F7
:1042D000232F342F452F5527892D9927AA27BB2710
:1042E000280F391F4A1F5B1FD401C3018070A070C3
:1042F000B070BA2FA92F982F8827280F391F4A1F6F
:104300005B1FB62DAA2799278827280F391F4A1F18
:104310005B1F2093FB013093FC014093FD01509300
:10432000FE0188859985AA85BB858093F7019093C6
:10433000F801A093F901B093FA01C2018896292FE0
:104340003327982F8827280F391F3093E2012093B5
:10435000E10186E08093E801488159816A817B818F
:1043600081ED91E00E949A1E1092040210920302C5
:104370008091E1019091E201782F6627892F99279A
:10438000680F791F685F7F4F8091DF0190E08F7029
:104390009070880F991F880F991F681B790B6250C6
:1043A00070409B0140E050E06E5F7F4F8BEE91E0EC
:1043B0000E94541E292F3327982F8827280F391F32
:1043C000309304022093030261ED71E0C201C696AE
:1043D0000E94A92F188ADF91CF911F910F91FF9012
:1043E000EF90DF90CF90BF90AF909F908F907F9095
:1043F0006F905F904F9008958F929F92AF92BF926F
:10440000DF92EF92FF920F931F93CF93DF937B0185
:104410008C015A0149018BB78F7D8BBF20E030E0C2
:10442000D22E86E190E0289FE001299FD00D389F91
:10443000D00D1124CA58DB4F88819981AA81BB8194
:104440000097A105B105F1F4822F0E94B420E88203
:10445000F9820A831B83BD82AC829F828E8282EDA9
:1044600094E0A0E0B0E088879987AA87BB8789E2BB
:1044700099E0A0E0B0E08C879D87AE87BF878EE192
:104480008B8B06C0D3942F5F3F4F2530310541F60B
:104490002D2D30E086E190E0289FF001299FF00D5E
:1044A000389FF00D1124EA58FB4F82E0808B6D2D70
:1044B00080E090E00E94DE208BB780628BBFDF91AE
:1044C000CF911F910F91FF90EF90DF90BF90AF9031
:1044D0009F908F900895482F50E026E130E0429F52
:1044E000F001439FF00D529FF00D1124EA58FB4F4D
:1044F0002FEF3FEF328B218B91E1908B682F80E083
:1045000090E00E94DE2008957F928F929F92AF925A
:10451000BF92CF92DF92EF92FF920F931F93CF93B0
:10452000DF9340E050E0842E9924F401EE0FFF1F4A
:10453000EE0FFF1FE456FE4F0190F081E02D309703
:1045400009F450C22091F5013091F6014F5F5F4FA1
:10455000832F9927322F2227820F931FE817F907FD
:1045600011F72091000221FF97C024FF95C081ED33
:1045700091E00E94F91E4091F3015091F401609185
:10458000EB017091EC018091ED019091EE010E94A0
:104590002820682F853008F025C2282F30E086E1DA
:1045A00090E0289F4001299F900C389F900C112487
:1045B00086E794E0880E991E8EE1E4018B8BEC84F3
:1045C000FD840E851F858C859D85AE85BF852C85D8
:1045D0003D854E855F85AC84BD84CE84DF84E12E2D
:1045E000FF240027112780709070B070892F9A2FB8
:1045F000AB2FBB27E80EF91E0A1F1B1F0894E11CF6
:10460000F11C011D111D207040705070542F432F5C
:10461000322F2227E20EF31E041F151FDA2CCC24A2
:10462000BB24AA24EA0CFB1C0C1D1D1DA80197012C
:10463000207030705070232F342F452F5527812F35
:104640009927AA27BB27280F391F4A1F5B1FD801AC
:10465000C7018070A070B070BA2FA92F982F88273B
:10466000280F391F4A1F5B1F1E2D0027FF24EE2431
:104670002E0D3F1D401F511FF401248735874687AB
:10468000578780E1808B80E090E00E94DE2081E00F
:1046900090E09A8B898BA6C1223051F581ED91E093
:1046A0000E94F91E4091F3015091F4016091EB01D9
:1046B0007091EC018091ED019091EE010E94282013
:1046C000682F853008F08EC1282F30E086E190E019
:1046D000289FF001299FF00D389FF00D1124EA5812
:1046E000FB4F82E1808B80E090E00E94DE207AC167
:1046F0004091F3015091F4016091EB017091EC0154
:104700008091ED019091EE010E942820782EE4E046
:10471000E81708F07EC081ED91E00E94F91E8091BB
:10472000000280FD02C082FF5DC1272D30E086E1DE
:1047300090E0289FF001299FF00D389FF00D112483
:10474000EA58FB4FE484F5840685178584859585B2
:10475000A685B7852485358546855785A484B58487
:10476000C684D784E12EFF24002711278070907023
:10477000B070892F9A2FAB2FBB27E80EF91E0A1FA6
:104780001B1F0894E11CF11C011D111D20704070BD
:104790005070542F432F322F2227E20EF31E041F96
:1047A000151FDA2CCC24BB24AA24EA0CFB1C0C1DFC
:1047B0001D1DA8019701207030705070232F342FD9
:1047C000452F5527812F9927AA27BB27280F391F47
:1047D0004A1F5B1FD801C7018070A070B070BA2F4C
:1047E000A92F982F8827280F391F4A1F5B1F1E2DBE
:1047F0000027FF24EE242E0D3F1D401F511F24874C
:10480000358746875787808980FF93C080E1808BFA
:104810008BC081ED91E00E94F91E472D50E086E1AA
:1048200090E0489FE001499FD00D589FD00D112482
:10483000CA58DB4F888980FD03C0888982FF7DC00C
:10484000EC84FD840E851F858C859D85AE85BF8596
:104850002C853D854E855F85AC84BD84CE84DF8408
:10486000E12EFF240027112780709070B070892FEF
:104870009A2FAB2FBB27E80EF91E0A1F1B1F0894A7
:10488000E11CF11C011D111D207040705070542F4F
:10489000432F322F2227E20EF31E041F151FDA2C9E
:1048A000CC24BB24AA24EA0CFB1C0C1D1D1DA80152
:1048B0009701207030705070232F342F452F5527CB
:1048C000812F9927AA27BB27280F391F4A1F5B1F53
:1048D000D801C7018070A070B070BA2FA92F982F8F
:1048E0008827280F391F4A1F5B1F1E2D0027FF2412
:1048F000EE242E0D3F1D401F511F2C873D874E87F4
:104900005F87888980FF15C0880C991C880C991CCA
:104910008CE991E0880E991EF40122813381872D64
:10492000F901099580E1888B672D80E090E00E9475
:10493000DE20872D0E94B42055C0888983FF0BC0DC
:10494000888984FF08C089899A8901969A8B898B06
:1049500088E1888B3AC086E190E0489F9001499FAA
:10496000300D589F300D1124F901EA58FB4F808912
:1049700084FF0AC0F901E557FB4F808180FD04C028
:104980008081816080832EC086E190E0489FF001A5
:10499000499FF00D589FF00D1124DF01AA58BB4F1D
:1049A000ED01888984FF1EC0E557FB4F808180FFA1
:1049B00019C089899A898F5F9F4FA1F080E1888B08
:1049C00089899A8901969A8B898B880C991C880C05
:1049D000991C8CE991E0880E991EE401EA81FB8123
:1049E000872D0995DF91CF911F910F91FF90EF9047
:1049F000DF90CF90BF90AF909F908F907F90089561
:104A0000CF93DF93C0E0D0E086E190E0C89FF00153
:104A1000C99FF00DD89FF00D1124EA58FB4F8389F0
:104A2000882329F580819181A281B3810097A10516
:104A3000B10519F183E0838B84898F5F848B81506A
:104A4000863088F08BB78F7D8BBF84E1808B6C2F95
:104A500080E090E00E94DE208BB780628BBF8C2FBD
:104A60000E94B4200AC08C2F0E947B2006C083893C
:104A70008F3F19F083898150838B2196C530D105F2
:104A800019F6DF91CF910895AF92BF92CF92DF9246
:104A9000EF92FF920F931F937C01A3EFAA2EA1E048
:104AA000BA2E872F9927762F6627860F971F909308
:104AB000F4018093F301852F9927542F4427840F05
:104AC000951F9093F6018093F501C7010896492F31
:104AD0005527982F8827480F591F5093F801409366
:104AE000F701C7014C96492F5527982F8827480F63
:104AF000591F5093E2014093E10181E18093E80165
:104B00006EEDC62E6FEFD62ECA0CDB1CB901A801C4
:104B1000C6010E949A1E1092FA011092F90180912A
:104B2000E1019091E201782F6627892F9927680F7C
:104B3000791F685F7F4F8091DF0190E08F709070E8
:104B4000880F991F880F991F681B790B675F7F4F2C
:104B50009B0140E050E069507040C50108970E94F9
:104B6000541E292F3327982F8827280F391F309359
:104B7000FA012093F901B601C7018A960E94A92F74
:104B80001F910F91FF90EF90DF90CF90BF90AF906B
:104B90000895EF92FF920F931F934093F301209398
:104BA000F401F092F801E092F7011093FA010093FA
:104BB000F9011092F6011092F50120E034E53093EE
:104BC000E2012093E10121E02093E80101ED11E0F1
:104BD000AB01BC01C8010E949A1E8091E101909135
:104BE000E201692F7727982F8827680F791F809116
:104BF000DF0190E08F709070880F991F880F991FC8
:104C0000681B790B20E030E040E050E083EF91E05A
:104C10000E94541E292F3327982F8827280F391FC9
:104C20003093F6012093F501B80182E690E00E94EE
:104C3000A92F1F910F91FF90EF900895CF93DF93CD
:104C4000CFEDD1E08091DF019091E0018050914063
:104C500009F099C08091E1019091E201089709F073
:104C600092C08091E301863009F08DC08091E4010B
:104C7000843009F088C02091F7013091F80140910B
:104C8000F9015091FA018091690490916A04A09110
:104C90006B04B0916C04281739074A075B0709F0C9
:104CA00072C08091E5019091E601E1E080309E07BD
:104CB00009F064C00E944C1D4091ED015091EE013D
:104CC0006091EF017091F001CE010E970E941B1EC2
:104CD00088E096E09093DE018093DD016091ED0124
:104CE0007091EE018091EF019091F0010E94F91D09
:104CF000853009F1DE0140E050E090E09C01220F98
:104D0000331F280F391F220F331F220F331FF901C2
:104D1000E40FF51FE65DFB4F8081FD01828BFA01F8
:104D2000EF5CFA4F8081FD0180874F5F5F4F1196E6
:104D30004630510561F780E092E09F838E83809139
:104D4000ED019091EE01A091EF01B091F001888FFB
:104D5000998FAA8FBB8F8091690490916A04A0916A
:104D60006B04B0916C048E879F87A88BB98B61ED23
:104D700071E08CE390E00E94A92F05C08050924022
:104D800011F40E944C1DDF91CF910895EF92FF9294
:104D90000F931F938091DD019091DE0126E0883012
:104DA000920719F40E941E26ACC0089709F0A9C00A
:104DB0002091EF013091F0014091F1015091F20109
:104DC0008091690490916A04A0916B04B0916C0485
:104DD000281739074A075B0709F093C00E944C1D4A
:104DE0008091E801813009F082C08091F30188232D
:104DF000C1F0883009F085C0E090F701F090F8012B
:104E00000091F9011091FA016091EB017091EC01B0
:104E10008091ED019091EE0120E040E00E94C925D3
:104E200070C08091EB019091EC01A091ED01B091E7
:104E3000EE019070A070B070BF93AF939F938F936B
:104E40008FEE90E09F938F930E94B41B8091EB01B3
:104E50009091EC01A091ED01B091EE01892F90E0CD
:104E6000A0E0B0E0BF93AF939F938F938BEE90E061
:104E70009F938F930E94B41B8091EB019091EC0162
:104E8000A091ED01B091EE018A2F90E0A0E0B0E09A
:104E9000BF93AF939F938F9387EE90E09F938F93F1
:104EA0000E94B41B8091EB019091EC01A091ED0167
:104EB000B091EE018B2F9927AA27BB27BF93AF9301
:104EC0009F938F9383EE90E09F938F930E94B41BE8
:104ED00089ED90E09F938F930E94B41B8DB79EB78E
:104EE0004A960FB6F8949EBF0FBE8DBF0AC086309B
:104EF00011F40E9484228091E801813111F40E9412
:104F000057201F910F91FF90EF900895CF93DF935B
:104F10008091680481FF09C00E9400250E94BD1C89
:104F2000809168048D7F809368048091680480FD7F
:104F30000DC018C0BE0188E592E00E941A2FFC0146
:104F4000E253FE4F10820E94C62602C0C1EDD1E09E
:104F5000B29BF0CF809168048E7F809368048BB7FA
:104F600080628BBFDF91CF9108958F929F92AF9215
:104F7000BF92CF92DF92EF92FF920F931F93CF9346
:104F8000DF93CDB7DEB7AA970FB6F894DEBF0FBE9A
:104F9000CDBF4B015C011FE0C12ED12CCC0EDD1E1C
:104FA0008091710490917204A0917304B091740483
:104FB00085017401E822F9220A231B232091690448
:104FC00030916A0440916B0450916C0482239323C6
:104FD000A423B523E816F9060A071B0719F485016F
:104FE000740108C0E0906D04F0906E0400916F04AD
:104FF0001091700488E096E09E878D87B801A70124
:10500000CE0101960E941B1E8091690490916A0452
:10501000A0916B04B0916C04F60186879787A08BF2
:10502000B18BE08EF18E028F138FA1E3B5E08D91ED
:105030008087128A319625E0A733B207C1F720E0B6
:1050400031E0F6013183208388E090E0938382830E
:1050500086E0848384E0858337832683BE016F5F87
:105060007F4F8AE290E00E94A92FCC24C501B401B1
:105070000E94F91DD82EC801B7010E94F91D853084
:1050800020F0F4E0FD15A8F025C024E02D1510F562
:1050900090E0FC01EE0FFF1FE80FF91FEE0FFF1F5E
:1050A000EE0FFF1FE65DFB4F86829782A086B186DA
:1050B00011C080E090E000000196E7E280319E0799
:1050C000D1F70E948627C394F4E1CF1679F680E0E9
:1050D00090E002C081E090E0AA960FB6F894DEBF9F
:1050E0000FBECDBFDF91CF911F910F91FF90EF9039
:1050F000DF90CF90BF90AF909F908F9008950F93C7
:105100001F930E94032940EC58EA61E07AE58EE1A2
:1051100090E00E94791C6093690470936A04809304
:105120006B0490936C044FEF5FEF6FEF70E082E2DF
:1051300090E00E94791C60937104709372048093D4
:1051400073049093740440EC58EA61E071E086E2E5
:1051500090E00E94791C60936D0470936E048093BC
:105160006F04909370041092310580E280933205B1
:1051700088E18093330581EB8093340585E180934A
:1051800035058FE68093360586E191E09F938F93F6
:105190000E94B41B0E94F12F8DE091E09F938F93AA
:1051A0000E94B41B01ED11E0B8018CE390E00E9475
:1051B000A92FB8018CE390E00E94A92F80916C0484
:1051C00090E09F938F9380916B0490E09F938F93D7
:1051D00080916A0490E09F938F938091690490E09E
:1051E0009F938F9382EF90E09F938F930E94B41BC5
:1051F0008DB79EB70E960FB6F8949EBF0FBE8DBFAB
:105200001F910F9108958EB58D608EBD1DBC1CBC85
:1052100088E09DE39BBD8ABD89B7806189BF089501
:105220001F920F920FB60F9211242F933F934F931B
:105230005F936F937F938F939F93AF93BF93EF93FE
:10524000FF938091FB049091FC04A091FD04B09128
:10525000FE040196A11DB11D8093FB049093FC04F4
:10526000A093FD04B093FE048091C6019091C70104
:10527000A091C801B091C9010196A11DB11D8093F3
:10528000C6019093C701A093C801B093C9010197CB
:10529000A109B109815B9440A040B04050F0109248
:1052A000C6011092C7011092C8011092C9010E9454
:1052B0007F288091680482608093680480919801BF
:1052C0009091990101979093990180939801FF9192
:1052D000EF91BF91AF919F918F917F916F915F916E
:1052E0004F913F912F910F900FBE0F901F901895E7
:1052F000E0E0F0E009940895AC01809137059091C9
:105300003805892BA1F020E0E199FECFA22FB0E073
:10531000FD01EE0FFF1FE95CFA4F80819181A40F20
:10532000B51F082E0E947A3B2F5F243068F3089542
:105330000895EF92FF921F93CF93DF93C2E2D1E0E3
:1053400096EBE92E92E0F92EFE0121961491812F21
:1053500090E09F938F93FF92EF920E94B41B0F9067
:105360000F900F900F90112379F7DF91CF911F913C
:10537000FF90EF9008956F927F928F929F92AF92DD
:10538000BF92CF92DF92EF92FF920F931F936090A4
:10539000FB047090FC048090FD049090FE04E0906B
:1053A000FB04F090FC040091FD041091FE04609158
:1053B000FB047091FC048091FD049091FE042CE3A9
:1053C00030E040E050E00E94483B5B016C01BB24B0
:1053D000C801B7012CE330E040E050E00E94483BB8
:1053E000CA01B9012CE330E040E050E00E94483BA4
:1053F0007B018C01FF24C401B30120E13EE040E0C9
:1054000050E00E94483BCA01B90128E130E040E089
:1054100050E00E94483B70E0BF92AF92FF92EF9243
:105420007F936F9389EB92E09F938F930E94B41BBD
:105430008DB79EB708960FB6F8949EBF0FBE8DBF6E
:105440001F910F91FF90EF90DF90CF90BF90AF90A2
:105450009F908F907F906F900895E0913705F09125
:1054600038058091390590913A052AE731E0EE0F31
:10547000FF1FE20FF31F91838083E0913705F091C6
:105480003805EE0FFF1FE20FF31F808191812091FD
:105490003705309138059F938F933F932F938FEC6F
:1054A00092E09F938F930E94B41B8DB79EB7069690
:1054B0000FB6F8949EBF0FBE8DBF08952F923F92F6
:1054C0004F925F926F927F928F929F92AF92BF9214
:1054D000CF92DF92EF92FF920F931F93CF93DF93C0
:1054E000C0E0D0E090E2292E93E0392E87E1482EEB
:1054F00083E0582E02E1602E03E0702E1DE0812E25
:1055000013E0912EB8E0AB2EB3E0BB2EADEFCA2E68
:10551000A2E0DA2EF0EFEF2EF2E0FF2EDF93CF9332
:105520003F922F920E94B41B86E190E0C89F8001B9
:10553000C99F100DD89F100D11240A581B4FF80158
:1055400080819181A281B3819070A070B070BF936F
:10555000AF939F938F935F924F920E94B41BF80179
:1055600080819181A281B381892F90E0A0E0B0E099
:10557000BF93AF939F938F937F926F920E94B41BC0
:10558000F80180819181A281B3818A2F90E0A0E00F
:10559000B0E0BF93AF939F938F939F928F920E949F
:1055A000B41BF80180819181A281B3818B2F99274F
:1055B000AA27BB27BF93AF939F938F93BF92AF92BE
:1055C0000E94B41BF8012481358184819581892F43
:1055D0009927322F2227820F931F9F938F93DF9259
:1055E000CF920E94B41BF80183892DB73EB7205E8D
:1055F0003F4F0FB6F8943EBF0FBE2DBF90E09F9374
:105600008F93FF92EF920E94B41B21960F900F9000
:105610000F900F90C530D10509F080CFDF91CF9169
:105620001F910F91FF90EF90DF90CF90BF90AF90C0
:105630009F908F907F906F905F904F903F902F90B2
:1056400008952F923F924F925F926F927F928F9226
:105650009F92AF92BF92CF92DF92EF92FF920F9301
:105660001F93CF93DF93C0E0D0E0BEE42B2EB3E0D6
:105670003B2EA9E44A2EA3E05A2EF0E46F2EF3E06D
:105680007F2EEBE38E2EE3E09E2E76E3A72E73E0D3
:10569000B72E61E3C62E63E0D62E54E2E52E53E02A
:1056A000F52E8E01000F111F0C0F1D1F000F111F73
:1056B000000F111F065D1B4FF801808190E09F9342
:1056C0008F93DF93CF9322E633E03F932F930E9493
:1056D000B41BF801818190E09F938F932DE533E017
:1056E0003F932F930E94B41BF801828190E09F9317
:1056F0008F9328E533E03F932F930E94B41BF8016A
:10570000838190E09F938F9323E533E03F932F9322
:105710000E94B41BF801848190E09F938F933F9285
:105720002F920E94B41BF801858190E09F938F9384
:105730005F924F920E94B41BF80186819781A085E9
:10574000B1859070A070B070BF93AF939F938F930B
:105750007F926F920E94B41BF80186819781A08589
:10576000B1852DB73EB7205E3F4F0FB6F8943EBFD0
:105770000FBE2DBF892F90E0A0E0B0E0BF93AF93A4
:105780009F938F939F928F920E94B41BF801868102
:105790009781A085B1858A2F90E0A0E0B0E0BF930B
:1057A000AF939F938F93BF92AF920E94B41BF80167
:1057B00086819781A085B1858B2F9927AA27BB2742
:1057C000BF93AF939F938F93DF92CF920E94B41BAE
:1057D000F801828593859F938F93FF92EF920E94A9
:1057E000B41B21962DB73EB72A5E3F4F0FB6F894F3
:1057F0003EBF0FBE2DBFC530D10509F052CFDF919E
:10580000CF911F910F91FF90EF90DF90CF90BF90BD
:10581000AF909F908F907F906F905F904F903F9050
:105820002F9008958091730590E09F938F938FE65A
:1058300093E09F938F930E94B41B0F900F900F9053
:105840000F9008958091360590E09F938F938091FB
:10585000350590E09F938F938091340590E09F935E
:105860008F938091330590E09F938F9380913205C1
:1058700090E09F938F938091310590E09F938F9359
:1058800087E893E09F938F930E94B41B8DB79EB7D8
:105890000E960FB6F8949EBF0FBE8DBF0895AF92BF
:1058A000BF92CF92DF92EF92FF920F931F9380915E
:1058B000370590913805892BF1F1E0903705F0908C
:1058C0003805A0903905B0903A0580913B0590913C
:1058D0003C0520913D0530913E05CC24DD24DC2C97
:1058E000CB2CBA2CAA24A0E0B0E0DC0199278827B1
:1058F000A80EB91ECA1EDB1E00E010E0AE0CBF1CD5
:10590000C01ED11E40E050E0522F442733272227EB
:10591000A20EB31EC41ED51EC601B5010E94B52736
:1059200011E0E12EF12C01E010E020E048E0C6019A
:10593000B5010E94C9251F910F91FF90EF90DF9054
:10594000CF90BF90AF9008950E943137089586E2BE
:1059500090E00E947C2940EC58EA61E071E086E228
:1059600090E00E94791C60936D0470936E048093A4
:105970006F04909370048091700490E09F938F93D4
:1059800080916F0490E09F938F9380916E0490E0DC
:105990009F938F9380916D0490E09F938F9389EAFA
:1059A00093E09F938F930E94B41B8DB79EB70A9686
:1059B0000FB6F8949EBF0FBE8DBF089582E290E0AF
:1059C0000E947C294FEF5FEF6FEF70E082E290E082
:1059D0000E94791C60937104709372048093730425
:1059E000909374048091740490E09F938F938091BE
:1059F000730490E09F938F938091720490E09F9343
:105A00008F938091710490E09F938F9386EC93E045
:105A10009F938F930E94B41B8DB79EB70A960FB6C3
:105A2000F8949EBF0FBE8DBF089582E390E00E9460
:105A30007C294DE455E266E07BE382E390E00E943E
:105A4000791C6093CD017093CE018093CF01909328
:105A5000D0018091D00190E09F938F938091CF01EE
:105A600090E09F938F938091CE0190E09F938F93CE
:105A70008091CD0190E09F938F9381EE93E09F936F
:105A80008F930E94B41B8DB79EB70A960FB6F894F9
:105A90009EBF0FBE8DBF08958EE190E00E947C29CD
:105AA00040EC58EA61E07AE58EE190E00E94791CD2
:105AB0006093690470936A0480936B0490936C0400
:105AC00080916C0490E09F938F9380916B0490E0A1
:105AD0009F938F9380916A0490E09F938F9380911E
:105AE000690490E09F938F938FEF93E09F938F9340
:105AF0000E94B41B8DB79EB70A960FB6F8949EBF4E
:105B00000FBE8DBF0895AF92BF92CF92DF92EF92FA
:105B1000FF920F931F93CF93DF93CDB7DEB72297FA
:105B20000FB6F894DEBF0FBECDBF9A83898364E6BB
:105B300070E0CE0101960E94EE3A6C01FF2410C085
:105B4000F394EF2DF0E0EE0FFF1FEE0FFF1FE55572
:105B5000FF4F80819181892B19F480E090E03FC054
:105B60000F2D10E0F801EE0FFF1FEE0FFF1FE555A0
:105B7000FF4FB601808191810E94743A892B01F711
:105B8000EE24FF24B6E6AB2EB0E0BB2E6E010894E7
:105B9000C11CD11CB501C6010E94EE3A40E050E0A4
:105BA00060E070E00E940639F701EE0FFF1FE95C2C
:105BB000FA4F718360830894E11CF11C8AE0E816B7
:105BC000F10441F7000F111F000F111F05551F4F62
:105BD000F80182819381FC01099581E090E0229691
:105BE0000FB6F894DEBF0FBECDBFDF91CF911F91EE
:105BF0000F91FF90EF90DF90CF90BF90AF900895FE
:105C0000CF93DF93DC01EB01AB0131C090E09695BF
:105C1000879596958795FE0181939F019C9193703E
:105C20009295907F9983FD018181882321F4E90178
:105C3000219622E020C082958F70890F8983FD0113
:105C400091819F70990F990F9A838281882319F40B
:105C5000239621E010C08295869586958370890FE2
:105C60008A83FD0182818F738B83249613968C9196
:105C7000882361F620E01882DA0108C0EC91F0E098
:105C8000EF73F070E85EFB4FE491ED93AC17BD0746
:105C9000A9F7FD01922F02C08DE381939150E0F7A7
:105CA000A20FB11D1C92DF91CF910895FC01C49801
:105CB0008AE38FB9779906C0FDCF1FB8779BFECFD7
:105CC0008FB18193615070408FEF6F3F7807A9F7D4
:105CD000C49A0895FC01C4988AE78FB9779BFECFD8
:105CE00081918FB961507040779BFECF611571052E
:105CF000B9F7C49A0895C498962F9F71982B9FB9AD
:105D0000779BFECF1FB8779BFECF67FF03C01FB8FE
:105D1000779BFECF8FB1C49A90E00895C4988FB955
:105D2000779BFECF6FB9779BFECFC49A0895FF9201
:105D30000F931F93F62E082F0F710B3198F4182F25
:105D4000107680917405181769F01093740563E05C
:105D50008FEB0E948E2E129516951770612F8FE98A
:105D60000E948E2E6F2D802F80640E948E2E1F9198
:105D70000F91FF9008950F931F93082F90E08F715C
:105D800090704B979CF4102F107680917405181723
:105D900069F01093740563E08FEB0E948E2E1295CC
:105DA00016951770612F8FE90E948E2E602F80E06C
:105DB0000E947B2E90E01F910F9108950F931F93E7
:105DC0008B01682F84ED0E94972E602F86ED0E9434
:105DD000972E012F1127602F87ED0E94972E8AEEB4
:105DE0000E94BB2E80FDFBCF1F910F9108950F9352
:105DF0001F93682F84ED0E94972E61E082ED0E9430
:105E0000972E8AEE0E94BB2E80FDFBCF60E082EDD4
:105E10000E94972E89ED0E94BB2E082F10E0102FB4
:105E2000002788ED0E94BB2E90E0802B912B1F91C4
:105E30000F910895EF92FF920F931F93CF93DF93EB
:105E4000EC017B018CE10E94BB2E86FD08C089E33A
:105E50000E94BB2E882319F400E010E072C060910C
:105E600075057091760580E00E94972E609175050A
:105E700070917605672F772781E00E94972E60E06A
:105E80008AE30E947B2E90E09093760580937505BF
:105E9000009175051091760560E08AE30E947B2EE3
:105EA00090E0982F8827802B912B909376058093F4
:105EB000750560E08AE30E947B2E082F10E060E009
:105EC0008AE30E947B2E90E0982F8827082B192BBD
:105ED00060E08AE30E947B2E60E08AE30E947B2ED2
:105EE000C017D10708F48E01B801C7010E94562ED1
:105EF0008091750590917605809175059091760554
:105F0000019780509A4130F06FEF8CE00E94972EFD
:105F100069E110C0609175057091760561508CE063
:105F20000E94972E609175057091760561507040C2
:105F3000672F77278DE00E94972E60E48EE90E94FC
:105F40008E2EC801DF91CF911F910F91FF90EF909E
:105F50000895EF92FF920F931F93CF93DF93EC017D
:105F60007B0100E010E08FE10E94BB2E83FF09C09F
:105F700080EA9FE00197F1F70F5F1F4F0233110591
:105F800091F760E082E00E94972E6AE183E00E9430
:105F9000972E6C2F86E00E94972EC050D64E6D2F04
:105FA0007727C050DA4187E00E94972E60E08AE7A9
:105FB0000E948E2EBE01C7010E946A2E60E88FE902
:105FC0000E948E2E60E88FEB0E948E2E6CE08FE98F
:105FD0000E948E2EDF91CF911F910F91FF90EF9035
:105FE0000895CF93DF938FEF80937405BC9AC49A82
:105FF000C79A87B3886B87BBBE9880E58DB981E06F
:106000008EB980E090E0A0E0B0E000000196A11D14
:10601000B11D80342DE0920723E0A20720E0B207F3
:10602000A1F76FEF8FEF0E948E2E80E090E0A0E04E
:10603000B0E000000196A11DB11D8034EDE09E0787
:10604000E3E0AE07E0E0BE07A1F7C0E0D0E001C0AA
:1060500021968DE10E94BB2E80FD04C0FDEFC83E5D
:10606000DF07B1F71092760510927505CBE5D4E005
:10607000FE0164912197FE0184910E94972E239640
:10608000F4E0C738DF07A1F760E071E080E10E942B
:10609000DE2E60EC8BE10E94972E64E08FE90E9477
:1060A0008E2E6AE477E384E10E94DE2E8FE10E9467
:1060B000BB2E8093730582E70E94BB2E80937305ED
:1060C000DF91CF91089590E02DE030E0A901849F09
:1060D0009001859F300D949F300D1124E3E9F5E088
:1060E000D901AE0FBF1F8C91887F8C933897E20F38
:1060F000F31F13821282118210828C91877F8C93FE
:1061000087E795E09583848380E791E09287818794
:1061100085E791E0948783878EE891E09783868373
:1061200008952F923F924F925F927F928F929F920B
:10613000AF92BF92CF92DF92EF92FF920F931F9395
:10614000CF93DF93CDB7DEB72A970FB6F894DEBFB3
:106150000FBECDBF782E882E99248DE090E0889ECA
:106160009001899E300D989E300D1124F901ED5655
:10617000FA4F808180FD07C0F901E557FA4F8BE7A0
:1061800092E39383828386E190E0889EF001899E6A
:10619000F00D989EF00D1124EA58FB4F808988235A
:1061A00039F4F901E557FA4F808191819383828315
:1061B000F901E557FA4F8281938191838083CC2442
:1061C000DD247F015E010894A11CB11C2BE9222E65
:1061D00022E3322E97EA492E92E3592EF7010281EB
:1061E0001381B8016F5F7F4F73836283F8018491DD
:1061F000F601EF52FE4F86AB853209F0F8C043E05E
:1062000050E08BEE90E00E944A3A892B99F50C5FA2
:106210001F4FF80184910F5F1F4FF80134913051E7
:106220002AE0829FC0011124380FE32FF0E0EE0F27
:10623000FF1FE658FE4F4AE050E0B5018081918192
:106240000E94063B6AE070E0C5010E94E33A082F15
:1062500010E0A801B501C601895F9D4F0E94623A16
:1062600001501040C00ED11EF70182819381059626
:1062700093838283F7010281138144E050E0B801E7
:106280008FEE90E00E944A3A892B09F044C00B5FE0
:106290001F4FF8013491305301501040F8016491C0
:1062A000623461F0633418F46134C1F405C06334BE
:1062B00039F0643499F406C02BB305C028B303C089
:1062C00025B301C022B381E090E002C0880F991F7E
:1062D0003A95E2F7282311F0B20102C065EA72E3B1
:1062E000C5010E94433A6AE070E0C5010E94E33AAA
:1062F000082F10E0A801B501C601895F9D4F0E94DB
:10630000623A01501040C00ED11EF7018281938184
:10631000069693838283F7010281138143E050E064
:10632000B80184EF90E00E944A3A892B09F044C0FA
:106330000C5F1F4FF8013491305301501040F801A9
:106340006491623461F0633418F46134C1F405C0BF
:10635000633439F0643499F406C029B305C026B318
:1063600003C023B301C020B381E090E002C0880FD6
:10637000991F3A95E2F7282311F0B10102C060E9B4
:1063800072E3C5010E94433A6AE070E0C5010E94D1
:10639000E33A082F10E0A801B501C601895F9D4FBF
:1063A0000E94623A01501040C00ED11EF701828156
:1063B0009381059693838283F7016281738143E021
:1063C00050E088EF90E00E944A3A892B81F486E100
:1063D00090E0889EF001899EF00D989EF00D1124AA
:1063E000EA58FB4F8DEF9FEF928B818B09C0089489
:1063F000C11CD11CFCE8CF16F1E0DF0608F4EECE9C
:1064000086E190E0889EF001899EF00D989EF00D47
:106410001124EA58FB4F88E1808B672DC6010E944A
:10642000DE202A960FB6F894DEBF0FBECDBFDF91F7
:10643000CF911F910F91FF90EF90DF90CF90BF9081
:10644000AF909F908F907F905F904F903F902F9054
:1064500008957F928F929F92AF92BF92CF92DF92D8
:10646000EF92FF920F931F93CF93DF93782E80913B
:10647000FF01082F10E0007F107015950795159506
:1064800007956FEA72E3C8018D509E4F0E94AC3AA7
:10649000892B81F0272D30E08DE090E0289FF001DE
:1064A000299FF00D389FF00D1124ED56FA4F808191
:1064B00088608083A72CBB248DE090E0A89ED0014B
:1064C000A99EB00DB89EB00D11245BE8E52E55E0F5
:1064D000F52EEA0EFB1EE701EE81FF818081882305
:1064E00009F45BC0B8016E5D7F4F8091E201282FF7
:1064F00030E02E5D3F4F8091E10190E0982F88279A
:10650000280F391F201B310BAB014F525E4FED019D
:10651000CD56DA4FD70187E7C82E85E0D82EFEE8A2
:10652000EF2EF1E0FF2E36C0888180FD19C0FA0100
:106530008081FD0184809580F40191914F01FD01DE
:1065400095828482891711F0D582C482FD018481ED
:106550009581FC018081882319F48881816088837A
:10656000FA018081FD0186809780F40191914F01AD
:10657000FD0197828682891711F0F782E682FD017C
:1065800086819781FC0180814F5F5F4F882329F0CE
:106590006F5F7F4F6217730738F28DE090E0A89E1F
:1065A000A001A99E500DB89E500D1124FA01ED5680
:1065B000FA4FE081E0FF98C0E3FF96C0B8016E5D3E
:1065C0007F4F8091E201282F30E02E5D3F4F809178
:1065D000E10190E0982F8827280F391F201B310BED
:1065E000EB01CF52DE4FDA01A557BA4F90E7E92E03
:1065F00091E0F92E85E7C82E81E0D82E71C09881F0
:10660000FD0181849284F40181914F01FD01928604
:106610008186981711F0F286E186FD0181849284CB
:10662000F40180818823C9F589818434F1F08534AF
:1066300038F4823491F08334A0F4813459F509C0E0
:106640008634D9F08634A8F08734D9F0883411F52F
:106650001CC08091CA018F5F1BC08091CA018E5FF0
:1066600017C08091CA018C5F13C08091CA01885FF6
:106670000FC08091CA01805F0BC08091CA01805E0B
:1066800007C08091CA01805C03C08091CA01805814
:106690008093CA01FD01F286E186FD018384948422
:1066A000F40181914F01FD0194868386981711F0C2
:1066B000D486C386FD0183859485FC018081219663
:1066C000882361F4FA01ED56FA4F8081877F808339
:1066D0008091CA0185BB1092CA0106C06F5F7F4FCF
:1066E0006217730708F48BCF8DE090E0A89EF0014D
:1066F000A99EF00DB89EF00D1124E557FA4F828146
:106700009381892B09F079C0F801B7968091E20155
:10671000282F30E02E5D3F4F8091E10190E0982FCF
:106720008827280F391F201B310BDF01AF52BE4FC6
:1067300016C08D918D3091F4EF52FE4F10828091F2
:10674000FF01C82FD0E0C07FD070D595C795D595F3
:10675000C795CD50DE4F00E010E03EC03196E21705
:10676000F30738F3ECCFB701CE010E94873A0F5FF1
:106770001F4F892B89F18DE090E0A89E4001A99ED2
:10678000900CB89E900C1124E401CD56DA4F18817C
:10679000126018836CEF70E0C7010E94873A61E0D5
:1067A00071E0C7010E94873A892B19F088818260C5
:1067B000888366E071E0C7010E94873A892B19F04F
:1067C00088818D7F8883F401E557FA4FE6018A813D
:1067D0009B819383828311C0C02EDD24CC0CDD1CF1
:1067E000CC0CDD1CE4E5F1E0CE0EDF1EF601E0800E
:1067F000F180E114F10409F0B6CF8DE090E0A89E9D
:106800009001A99E300DB89E300D1124D901A557D5
:10681000BA4FED01EE81FF818081882331F4F901C7
:10682000ED56FA4FE081E3FF17C086E190E0A89EA5
:106830008001A99E100DB89E100D11240A581B4FFF
:1068400080E1F801808B672D80E090E00E94DE20DF
:1068500081E090E0E8012FC0E0FD30C086E190E0EB
:10686000A89EE001A99ED00DB89ED00D1124CA5853
:10687000DB4F888983FF22C08BE792E3FD0193837E
:1068800082838091FF0190E0807F9070959587953D
:106890009595879541E850E069EF71E38D509E4FE3
:1068A0000E943A3A88E1888B672D81E890E00E9447
:1068B000DE2082E090E09A8B898B62C08DE090E0D0
:1068C000A89E9001A99E300DB89E300D1124F901AB
:1068D000E557FA4F82819381892B99F480918C013D
:1068E00090918D01019690938D0180938C0186E8A3
:1068F00094E093838283F901ED56FA4F80818D7F76
:10690000808386E190E0A89EE001A99ED00DB89E0C
:10691000D00D1124CA58DB4F82E090E09A8B898B0E
:10692000F901ED56FA4FE081E695E170E13071F43E
:106930008091FF0190E0807F907095958795959567
:10694000879547E550E061EA71E30FC0EE23C1F49B
:106950008091FF0190E0807F907095958795959547
:10696000879547E550E069E471E38D509E4F0E94A2
:106970003A3A88E1888B672D87E590E00E94DE2017
:10698000DF91CF911F910F91FF90EF90DF90CF900B
:10699000BF90AF909F908F907F900895EF92FF925D
:1069A0001F93CF93DF93182FE82EFF2486E190E00A
:1069B000E89EE001E99ED00DF89ED00D1124CA5842
:1069C000DB4F888980FD33C089899A89019719F442
:1069D000812F0E94633089899A89039720F4812F3F
:1069E0000E94293224C089899A89039748F08989AD
:1069F0009A898E5F9F4F20F4812F0E94913017C09B
:106A000086E190E0E89EF001E99EF00DF89EF00D21
:106A10001124EA58FB4F818992898E5F9F4F38F08D
:106A20008EEF9FEF928B818B812F0E946B22DF91E3
:106A3000CF911F91FF90EF90089567E775E08BE08D
:106A400091E00E94002E6EEC74E380E590E00E94DD
:106A5000E41C0895FF920F931F9360916000709162
:106A6000610080916604909167046817790709F4C2
:106A70006AC000E010E0F02E86E190E0089FF0018F
:106A8000099FF00D189FF00D1124EA58FB4F8681E5
:106A900097818050974109F047C08091FA0480FDAA
:106AA00052C08091FA0481608093FA048091620060
:106AB00090916300909367048093660440E050E0F7
:106AC00015C0FA01EF52FE4FD9018D9186ABB093FC
:106AD0006704A0936604A053B54031F420533040BE
:106AE00030936704209366044F5F5F4F20916604E4
:106AF000309167046217730721F786E190E0F8018F
:106B0000E89F8001E99F100DF89F100D11240A588D
:106B10001B4F88E1F801808B6F2DCA010E94DE2097
:106B200083E0F801838B0FC00F5F1F4F0530110505
:106B300009F0A1CF8091750482FF05C08091750492
:106B40008B7F809375041F910F91FF9008951F9381
:106B5000CF93DF93182FE82FF0E086E190E0E89FD5
:106B6000E001E99FD00DF89FD00D1124CA58DB4FEA
:106B7000888980FF06C0809175048B7F809375049F
:106B8000ABC089899A89892B21F089899A890197D3
:106B9000F1F481E090E09A8B898B46E150E064EB60
:106BA00072E387E092E00E943A3A612F86E190E03A
:106BB0000E94DE208091750484608093750480912A
:106BC000FA048E7F8093FA048FEF8B8B85C08989BE
:106BD0009A89029708F443C0888983FF40C082E005
:106BE00090E09A8B898B2091FF0130E0207F3070FC
:106BF0003595279535952795B9016E5D7F4F809125
:106C0000E201482F50E04E5D5F4F8091E10190E03E
:106C1000982F8827480F591F421B530BDB01AF5297
:106C2000BE4F06C05D9BFECF8D918CB96F5F7F4FCD
:106C300064177507BCF386E190E09F01289FF0017F
:106C4000299FF00D389FF00D1124EA58FB4F80E189
:106C5000808B612F80E090E00E94DE203DC086E1C5
:106C600090E0E89FD001E99FB00DF89FB00D11248E
:106C7000AA58BB4FED0189899A890297B8F0888993
:106C800084FF14C08091FA0480FF10C08FEF8B8BBB
:106C900080916604909167049093630080936200F2
:106CA0008091FA048E7F8093FA0416C086E190E00A
:106CB0009F01289FF001299FF00D389FF00D1124AE
:106CC000EA58FB4F8089882339F48091FA048E7F3B
:106CD0008093FA040E942A35DF91CF911F91089585
:106CE00067EA75E387E190E00E94E41C08956F92E3
:106CF0007F928F929F92AF92BF92CF92DF92EF924C
:106D0000FF920F931F9389E193E39F938F930E94C8
:106D1000B41BE0902302F090240200912502109110
:106D20002602212F332744275527D801C701807019
:106D30009070B070892F9A2FAB2FBB27280F391F67
:106D40004A1F5B1F205F314F4F4F5F4FD801C70174
:106D50008070A070B070BA2FA92F982F8827280FA5
:106D6000391F4A1F5B1F1E2D0027FF24EE242E0D06
:106D70003F1D401F511F2093230230932402409354
:106D80002502509326022093FB043093FC04409389
:106D9000FD045093FE046090FB047090FC0480900E
:106DA000FD049090FE04E090FB04F090FC04009140
:106DB000FD041091FE046091FB047091FC0480912D
:106DC000FD049091FE042CE330E040E050E00E948E
:106DD000483B5B016C01BB24C801B7012CE330E0E8
:106DE00040E050E00E94483BCA01B9012CE330E08A
:106DF00040E050E00E94483B7B018C01FF24C4012D
:106E0000B30120E13EE040E050E00E94483BCA016F
:106E1000B90128E130E040E050E00E94483B70E0DA
:106E2000BF92AF92FF92EF927F936F938FEF92E3B7
:106E30009F938F930E94B41B8DB79EB70A960FB68F
:106E4000F8949EBF0FBE8DBF1F910F91FF90EF90E2
:106E5000DF90CF90BF90AF909F908F907F906F907A
:106E60000895AF92BF92CF92DF92EF92FF920F936D
:106E70001F93CF93DF93E090CD01F090CE0100916E
:106E8000CF011091D001C801B7010E94B527813010
:106E900059F5CC24DD24CBECD2E3F3E9AF2EF1E0BD
:106EA000BF2EFE0121968491D601AF52BE4FFD0147
:106EB00082A744E050E0BE01C5010E944A3AF601B3
:106EC0003196892B29F06F0182E0EE32F80749F7FD
:106ED000980187014BE750E06CEF78E0CF010E940A
:106EE00044258CE493E302C08FE293E39F938F9356
:106EF0000E94B41B0F900F90DF91CF911F910F91C3
:106F0000FF90EF90DF90CF90BF90AF90089567E72C
:106F100076E38CEF98E00E94171D4DE455E266E0A1
:106F20007BE382E390E00E94791C6093CD01709333
:106F3000CE018093CF019093D00108958091E2011A
:106F400090E04C972091E10130E0322F2227820F10
:106F5000931F9F938F938AE693E39F938F930E944F
:106F6000B41B0F900F900F900F9008956EE977E388
:106F700089E591E00E94171D0895DF92EF92FF923C
:106F80000F931F938091CB019091CC01029778F0E1
:106F90008091CB019091CC01449748F48091CB0132
:106FA0009091CC0101969093CC018093CB0180917C
:106FB000CB019091CC01892B09F087C08EE894E336
:106FC0009F938F930E94B41B64EA78E382E399E075
:106FD0000E94E41C61ED72EA8AEB9CE30E94B527F3
:106FE0000F900F90882309F46AC080E090E0A0E041
:106FF000B0E000000196A11DB11D803824E8920781
:107000002EE1A20720E0B207A1F729E032E340E039
:1070100050E561ED72EA8AEB9CE30E94FC2185E079
:10702000E82EF12C012D112DDD241DC040E050E58E
:1070300061ED72EA8AEB9CE30E9428209FE1D91659
:1070400039F482E694E39F938F930E94B41B74C03B
:10705000E82EFF2400E010E025E0E216F10401052F
:10706000110580F0D39486E190E0E89EF001E99E5E
:10707000F00DF89EF00D1124EA58FB4F818992899A
:107080000197A1F68CE394E39F938F930E94B41B26
:1070900086E190E0E89EF001E99EF00DF89EF00D8B
:1070A0001124E557FB4F80818160808382E090E06E
:1070B0009093CC018093CB010F900F9006C081E09C
:1070C00090E09093CC018093CB018091CB01909183
:1070D000CC010B9798F18091CB019091CC01449712
:1070E00068F584E294E39F938F930E94B41B40E081
:1070F00050E561ED72EA8AEB9CE30E942820D82ECD
:10710000E82EFF244AE950E069E873E387E092E063
:107110000E943A3A86E190E0E89EF001E99EF00D87
:10712000F89EF00D1124EA58FB4F88E1808B6D2DFD
:107130008AE990E00E94DE200F900F901F910F913E
:10714000FF90EF90DF900895DF92EF92FF920F9300
:107150001F93CF93DF93D82E8091FF01C82FD0E0EB
:10716000C07FD070D595C795D595C795A2968E014D
:107170000F521E4F6CE9E62E64E3F62E0FC0F801A5
:1071800081918F0190E09F938F93FF92EF920E94E5
:10719000B41B21960F900F900F900F902091E20159
:1071A00030E02E5D3F4F8091E10190E0982F8827DD
:1071B000280F391F8091FF0190E0807F9070959596
:1071C000879595958795281B390BC217D307BCF275
:1071D0002D2D30E086E190E0289FF001299FF00DF1
:1071E000389FF00D1124EA58FB4F8FEF838B80E11D
:1071F000808B6D2D80E090E00E94DE20DF91CF91AA
:107200001F910F91FF90EF90DF900895A0E0B0E004
:10721000ECE0F9E30C94BD3B8C012B01EA01611514
:10722000710519F0FB0191838083209749F0CE010D
:107230000297839728F060E070E080E090E0F7C06C
:10724000F801E1908F018E2D90E00E946A3B892B1E
:10725000B9F7FDE2EF1631F4F801E1908F01332424
:10726000339407C0FBE2EF1619F4F801E1908F01A7
:107270003324209719F0C031D105E1F4F0E3EF1683
:1072800079F4F8018081883711F0883549F4F801E4
:10729000E1800E5F1F4FF2E03F2AC0E1D0E00AC05C
:1072A000209741F480E3E81619F4C8E0D0E002C06A
:1072B000CAE0D0E0C830D10571F0C930D10524F45E
:1072C000C230D10519F50DC0CA30D10581F0C031E9
:1072D000D105E1F415C0A12CB12CC12CB0E1DB2EFD
:1072E00022C0A12CB12CC12CA0E4DA2E1CC0FCECD5
:1072F000AF2EFCECBF2EFCECCF2EFCE0DF2E13C03B
:10730000A12CB12CC12CE8E0DE2E0DC09E0144273B
:1073100037FD4095542F60E070E080E090E80E94D7
:10732000483B59016A0120E030E040E050E060E075
:107330003E01882477FC8094982C70EDF72EFE0C8B
:10734000E9E0EF1570F48E2D81548A3118F499EC30
:10735000F92E06C08E2D81568A3150F589EAF82E15
:10736000FE0C8F2D90E08C179D0714F567FD1CC057
:10737000A216B306C406D506B0F0CA01B901A4012D
:1073800093010E94893B9B01AC012F0D311D411DD2
:10739000511D2130F0E03F07F0E04F07F0E85F07B4
:1073A00010F461E001C06FEFF801E1908F01C5CFEB
:1073B0004114510481F0662331F001501040F20174
:1073C0001183008308C031FE1AC002501040F20140
:1073D0001183008314C067FF12C030FE05C020E097
:1073E00030E040E050E804C02FEF3FEF4FEF5FE7A1
:1073F00082E290E09093CD058093CC0516C030FEDC
:1074000008C050954095309521953F4F4F4F5F4FA5
:107410000CC057FF0AC082E290E09093CD058093A4
:10742000CC052FEF3FEF4FEF5FE7CA01B901E1E174
:10743000CDB7DEB70C94D93BFC0188279927E89497
:1074400021912032E9F3293010F02E30C8F32B328D
:1074500041F02D3239F4689404C00E94273B820F1A
:10746000911D219120532A30C0F31EF490958195EF
:107470009F4F0895FB01DC0102C005900D92415021
:107480005040D8F70895FB01DC0105900D920020D3
:10749000E1F70895FB01DC014150504088F08D91E7
:1074A00081341CF08B350CF4805E659161341CF0E6
:1074B0006B350CF4605E861B611171F3990B0895B6
:1074C000881BFCCF6817790768F4FB01DC01E40F27
:1074D000F51FA40FB51F02C002900E9241505040FC
:1074E000D8F708950C942F3BFB01DC018D9181347A
:1074F0001CF08B350CF4805E619161341CF06B35AF
:107500000CF4605E861B611189F3990B0895FB01F1
:1075100051915523B1F0BF01DC01052E4D9144235B
:1075200069F010D0D9F7CD010190002049F04D91BC
:10753000411108D0C9F3FB014111EECF81E090E089
:1075400001970895402539F0403229F440294B57DE
:10755000465E08F018940895FB0155915523B1F04B
:10756000BF01DC01052E4D91442369F010D0D9F7FD
:10757000CD010590002049F04D91411108D0C9F38B
:10758000FB014111EECF81E090E001970895402585
:1075900039F0403229F440294B57465E08F01894E0
:1075A0000895FB01DC010D900020E9F7119701908F
:1075B0000D920020E1F70895FB01DC0101900D928E
:1075C0000020E1F70895FC01615070400190011026
:1075D000D8F7809590958E0F9F1F0895FC01A0818C
:1075E000B181AD01109681F03D91FB010190031630
:1075F0000110E1F7C9F7002011F4D00102C01E927A
:107600001196FC01A083B183CA010895FB019F017B
:10761000E8944230C4F04532B4F44A3029F497FB80
:107620001EF4909581959F4F642F77270E94A83B69
:10763000805D8A330CF0895D8193CB010097A1F7BF
:1076400016F45DE251931082C9010C94383B7AE044
:10765000979F902D879F802D910D11240895FB01F8
:10766000DC0102C001900D9241505040D8F70895BE
:10767000DC01FC01672F71917723E1F7329704C099
:107680007C916D9370836291AE17BF07C8F3089524
:10769000A1E21A2EAA1BBB1BFD010DC0AA1FBB1F16
:1076A000EE1FFF1FA217B307E407F50720F0A21B88
:1076B000B30BE40BF50B661F771F881F991F1A94F5
:1076C00069F760957095809590959B01AC01BD011F
:1076D000CF01089591111AC0803219F08950855058
:1076E000D0F70895E199FECFBFBBAEBBE09A1196EB
:1076F0000DB20895E199FECFBFBBAEBB0DBA119696
:107700000FB6F894E29AE19A0FBE08959927882758
:107710000895629FD001739FF001829FE00DF11DDB
:10772000649FE00DF11D929FF00D839FF00D749FFB
:10773000F00D659FF00D9927729FB00DE11DF91FA7
:10774000639FB00DE11DF91FBD01CF011124089504
:10775000AA1BBB1B51E107C0AA1FBB1FA617B70777
:1077600010F0A61BB70B881F991F5A95A9F7809593
:107770009095BC01CD0108952F923F924F925F9258
:107780006F927F928F929F92AF92BF92CF92DF9231
:10779000EF92FF920F931F93CF93DF93CDB7DEB796
:1077A000CA1BDB0B0FB6F894DEBF0FBECDBF09942A
:1077B0002A88398848885F846E847D848C849B8481
:1077C000AA84B984C884DF80EE80FD800C811B818F
:1077D000AA81B981CE0FD11D0FB6F894DEBF0FBEBE
:0877E000CDBFED010895FFCFBC
:1077E800FF04FF0420002E2C20005245534554006E
:1077F80041525000544350004950004E45540052E5
:107808004F55544552004E5450004D414300564583
:10781800520053560054494D45004E5450520050A2
:10782800494E470048454C50003F006A007829708F
:1078380000212B74005E2A78004C2D7B00DE2C7F03
:1078480000A72C8600152D8A00222C8E00122C925F
:10785800002D2A9500BB299A00A42C9F004F2CA428
:10786800009929A9009929000000005641400050BC
:107878004F52540050494E00454E44002E6A7067DE
:10788800002E676966002E68746D0061646D696E0C
:107898003A74696D00696E6465782E68746D00537A
:1078A80074617475732E68746D0063616D657261BF
:1078B8002E6A70670062616C6B652E676966006C82
:1078C80065646F6E2E676966006C65646F66662E08
:1078D80067696600150186041F01F8132A011B1A3F
:1078E8003501D2193F012B164901FF17000000008E
:1078F8004F55543D005355423D000A0032001E00CA
:1079080000000000000000000000000000000D0A58
:0A7918000D0A0025454E44007404DA
:00000001FF
